:090000000217DB0248B025730071
:10000B000249E6E4FFFE120731600C0FEF70010EA0
:0F001B0009E970F20A80EF220249F55322E02230
:07002B00024FFE43EA4022F0
:100033000241569000E27406F09000E07400F090E4
:1000430000E27412F07581AA1238050217DB75A855
:10005300009000E27406F09000E07480F09000E2FB
:10006300740CF00217DB244750524D430000020486
:1000730037E86480F8E933E83360110460F0ED3366
:10008300EC337009E8FCE9FDEAFEEBFF220460DED5
:10009300D3EB9FEA9EE99DE8C2E78CF0C2F795F0A7
:1000A300400CE8CCF8E9CDF9EACEFAEBCFFB120429
:1000B3000285D0F05804700320D5B3E804700750CC
:1000C30002B2D502044192D5EC0460F7E4CCC0E05F
:1000D300C398F8603B94186008400DD0E0FB02041D
:1000E30019E4FBFAC9FC8028E830E406E4C9FBE420
:1000F300CAFCE830E305E4C9CACBFCE85407601046
:10010300F8C3E913F9EA13FAEB13FBEC13FCD8F188
:1001130030F52FC3E49CFCEF9BFFEE9AFEED99FDB7
:10012300D0E0FBEF4E4D4C701222DB0302043EEC99
:100133002CFCEF33FFEE33FEED33FDED30E7EB0246
:100143000419EF2BFFEE3AFEED39FDD0E0FB50131F
:100153000BBB0003020441ED13FDEE13FEEF13FF8F
:10016300EC13FC020419EC4D6011E8497017ED33F0
:10017300EC3304600DE4FCFFFEFD22E933E83304B5
:1001830070F802043712040258046009E4CC248195
:10019300500628500902044128400302043EC0E0EF
:1001A300EB4A7044B98006D0E0FB02042DEF4E7099
:1001B3001CBD8008EBFFEAFEE9FD80EBE98DF0A4AE
:1001C300FEE5F0020252E9CDF9EAFEEBFFEF89F01A
:1001D300A4FCE5F0CE89F0A42EFFE435F0CD89F040
:1001E300A42DFEE435F08067EF4E7005BD80D78007
:1001F300C3EF8BF0A4ACF0EE8BF0A42CFCE435F051
:10020300F8EF8AF0A42CE5F038FCE433CB8DF0A4AE
:100213002CFCE5F03BF8EE8AF0A42CFCE5F038F872
:10022300E433CF89F0A42CFCE5F038CF3400CE8939
:10023300F0A42FFFE5F03EFEE433C98DF0A42EFEBB
:10024300E5F039CD8AF0A42FFFE5F03EFEE43DFD55
:1002530033D0E0FB50070BBB000F020441EC2CFC36
:10026300EF33FFEE33FEED33FD020419020441ECDC
:100273005D046005E8590470030204371204025850
:100283000460F6EC4860F2EC7004FDFEFF22C860E7
:10029300DB2481C85009C3986002500602043E98CB
:1002A30050CAF582E9294B4A7005AB8202042D75C9
:1002B300F0007C1A7880C3EF9BEE9AED99400DC352
:1002C300EF9BFFEE9AFEED99FDE842F0DC23ACF0E4
:1002D300D0E0FFD0E0FED0E0FDAB8220E7101BEBC7
:1002E30060BAEC2CFCEF33FFEE33FEED33FD02047A
:1002F30019E803F830E705C0F075F000EF2FFFEEC3
:1003030033FEED33FD40B830E7C280AA74F8CC6405
:1003130080CCC86480C8F582046043C3EB9FF5F0CA
:10032300EA9E42F0E99D42F0E89C45F060305018A7
:10033300E5825FFFE582F42B5582FB50210ABA0068
:100343001D09B90019088016E5825BFBE582F42FCD
:100353005582FF50090EBE00050DBD00010CC3EB15
:100363009FF5F0EA9E42F0E99D42F0E89C45F0607B
:1003730007CC4820E701B3EC22ED33EC33600A04E9
:100383007003BD8004ECB2E7FC2275F020800E758B
:10039300F010800575F0087D007E007F003392D554
:1003A30030D503120959EC334010EF33FFEE33FE1F
:1003B300ED33FDEC33FCD5F0ED22E5F0247EA2D540
:1003C30013CC92E7CDCEFF22EDD2E7CD33EC3392BF
:1003D300D524814006E4FFFEFDFC22FCE4CFCECD14
:1003E300CC24E0501174FF80EDC3CC13CCCD13CDDE
:1003F300CE13CECF13CF0470F030D5DE020959E906
:10040300D2E7C933E833F892D5EDD2E7CD33EC33F5
:10041300FC5002B2D522EC30E7100FBF000C0EBE29
:1004230000080DBD00040BEB6014A2D5EB13FCED2B
:1004330092E7FD2274FFFCFDFEFF22E480F8A2D5C3
:1004430074FF13FC7D80E480EFC0E0EFFBEEFAED78
:10045300F9ECF8120169D0E0F5F0EFFBEEFAEDF9F3
:10046300ECF8120997A3A3A3A3E8C0E0E9C0E0EA6C
:10047300C0E0EBC0E0C0F01201691209B4A3A3A36A
:10048300A3120078D0F0D0E0FBD0E0FAD0E0F9D0AE
:10049300E0F8D5F0D4223F8000004120000042C89C
:1004A3000000447A0000461C400047C350004974D2
:1004B30024004B1896804CBEBC205A0E1BCA6753AF
:1004C300C21C749DC5AEFB60065407601C23231237
:1004D30004F7EB543860091204E31204F2120169C1
:1004E300ECF8EDF9EEFAEFCB22EB1204F280F154C3
:1004F3003803241C900499FE93FC0EEE93FD0EEE3C
:10050300930ECE93FF22F920E72824F950037907AD
:10051300E4F42402FB18DBFDE624FB5014E9600D30
:10052300E4F618E604F6B40A08E4F6D9F57401F61D
:100533000A22C2D522ED33EC3392D5FA602AB4FFF6
:1005430033EDC2E77BFF60067A05795DE4227A0525
:10055300796620D5047A057961224E614E002B49D4
:100563004E46002D494E4600E47A08F608DAFC7B35
:1005730000740722E8C0E0ECC0E0EDC0E0EEC0E0AC
:10058300EFC0E0EA75F010A4CAABF075F04DA42BF0
:10059300FBE435F0FCEA2410FAEB34C5FBEC34D968
:1005A300FCEDC2E7FF75F056A4F42411C5F0F43452
:1005B300C58FF0A42AE5F03BE43CF620E7141204CF
:1005C300C9D0E0FFD0E0FED0E0FDD0E0FC12027223
:1005D3008014F4041204C9D0E0FFD0E0FED0E0FDA3
:1005E300D0E0FC120169D0E0F8E6FAEDD2E7CD33B2
:1005F300EC332482FBE4C3CF33CFCE33CECD33CD24
:1006030033DBF37B0775F00A846004F6081B0AE505
:10061300F0F6088FF0740AA4FFACF08EF0740AA40D
:100623002CFEACF050010C8DF0740AA42CFDE435C3
:10063300F0F608DBDE740722E709F608DFFA8046E6
:10064300E709F208DFFA803E88828C83E709F0A38A
:10065300DFFA8032E309F608DFFA8078E309F2086B
:10066300DFFA807088828C83E309F0A3DFFA806469
:1006730089828A83E0A3F608DFFA805889828A8315
:10068300E0A3F208DFFA804C80D280FA80C680D4DF
:10069300806980F28033801080A680EA809A80A8E7
:1006A30080DA80E280CA803389828A83ECFAE49319
:1006B300A3C8C582C8CCC583CCF0A3C8C582C8CCA7
:1006C300C583CCDFE9DEE7800D89828A83E493A3C7
:1006D300F608DFF9ECFAA9F0EDFB2289828A83ECB4
:1006E300FAE0A3C8C582C8CCC583CCF0A3C8C58231
:1006F300C8CCC583CCDFEADEE880DB89828A83E469
:1007030093A3F208DFF980CC88F0EF60010E4E600E
:10071300C388F0ED2402B4040050B9F582EB24023F
:10072300B4040050AF232345822390068B73BB018F
:100733000689828A83E0225002E722BBFE02E3227B
:1007430089828A83E49322BB010CE58229F582E541
:10075300833AF583E0225006E92582F8E622BBFEC0
:1007630006E92582F8E222E58229F582E5833AF556
:1007730083E49322BB010689828A83F0225002F725
:1007830022BBFE01F322EF8DF0A4A8F0CF8CF0A4DE
:1007930028CE8DF0A42EFE22BC000BBE0029EF8DC7
:1007A300F084FFADF022E4CCF875F008EF2FFFEEF4
:1007B30033FEEC33FCEE9DEC984005FCEE9DFE0F02
:1007C300D5F0E9E4CEFD22EDF8F5F0EE8420D21C5D
:1007D300FEADF075F008EF2FFFED33FD40079850A5
:1007E30006D5F0F222C398FD0FD5F0EA22C2D5EC6C
:1007F30030E709B2D5E4C39DFDE49CFCEE30E71578
:10080300B2D5E4C39FFFE49EFE12079BC3E49DFDA4
:10081300E49CFC800312079B30D507C3E49FFFE4ED
:100823009EFE22A3F8E0C5F025F0F0E58215827064
:10083300021583E0C838F0E822E88FF0A4CC8BF0EF
:10084300A42CFCE98EF0A42CFC8AF0EDA42CFCEA89
:100853008EF0A4CDA8F08BF0A42DCC3825F0FDE9C3
:100863008FF0A42CCD35F0FCEB8EF0A4FEA9F0EBB9
:100873008FF0A4CFC5F02ECD39FEE43CFCEAA42DC5
:10088300CE35F0FDE43CFC2275F008758200EF2FB5
:10089300FFEE33FECD33CDCC33CCC58233C5829B43
:1008A300ED9AEC99E58298400CF582EE9BFEED9A69
:1008B300FDEC99FC0FD5F0D6E4CEFBE4CDFAE4CC05
:1008C300F9A88222B800C1B90059BA002DEC8BF007
:1008D30084CFCECDFCE5F0CBF97818EF2FFFEE33C4
:1008E300FEED33FDEC33FCEB33FB10D703994004EF
:1008F300EB99FB0FD8E5E4F9FA227818EF2FFFEE16
:1009030033FEED33FDEC33FCC933C910D7059BE946
:100913009A4007EC9BFCE99AF90FD8E0E4C9FAE4A2
:10092300CCFB2275F010EF2FFFEE33FEED33FDCC41
:1009330033CCC833C810D7079BEC9AE899400AED2B
:100943009BFDEC9AFCE899F80FD5F0DAE4CDFBE4D3
:10095300CCFAE4C8F922C3E49FFFE49EFEE49DFDC4
:10096300E49CFC22EB9FF5F0EA9E42F0E99D42F005
:10097300E89C45F022E8600FECC313FCED13FDEE99
:1009830013FEEF13FFD8F122E6FC08E6FD08E6FEAE
:1009930008E6FF22E493FC740193FD740293FE7452
:1009A3000393FF22E6FB08E6F908E6FA08E6CBF82C
:1009B30022E493F8740193F9740293FA740393FB9A
:1009C30022ECF608EDF608EEF608EFF622ECF0A3BB
:1009D300EDF0A3EEF0A3EFF022A42582F582E5F07B
:1009E3003583F58322FAE6FB0808E6F925F0F618C5
:1009F300E6CA3AF622D083D082F8E49370127401E7
:100A030093700DA3A393F8740193F5828883E47321
:100A13007402936860EFA3A3A380DF8A838982E4CF
:100A230073EF4E6012EF60010EEDBB010B89828AFA
:100A330083F0A3DFFCDEFA2289F05007F709DFFC1D
:100A4300A9F022BBFEFCF309DFFCA9F022E5602438
:100A53004CF8E60560227849302F02784CE475F0B3
:100A6300011209E80207312028EB7F2ED2288018D3
:100A7300EF540F2490D43440D4FF302C0BEF24BF19
:100A8300B41A0050032461FFE56160021561056437
:100A9300E56470020563302F0D7849E475F00112A7
:100AA30009E8EF0207770219EB7403D22F8003E4FE
:100AB300C22FF5608B498A4A894BE4F561F563F5EA
:100AC30064E56160077F20120A8B80F57562FFC2BF
:100AD30029C228C22AC22BC22DC22EC230120A59E1
:100AE300FF700D302F057F00120A9CAF64AE6322A6
:100AF300B4255FC2D5C22C120A59FF24D0B40A0010
:100B0300501A75F00A786130D50508B6FF0106C69C
:100B1300A426F620D5047002D22B80D924CFB41A90
:100B230000EF5004C2E5D22C020D89D22980C6D22F
:100B33002880C0D22A80BCD2D580BAD22D80B47F7F
:100B430020120A8B202A077401B5610040F1120AB2
:100B530050FF120A8B020AC4D230D22E8095120A99
:100B630050FB120A50FA120A50F94A4B7006798068
:100B73007A0E7BFF202A2EE561602A7E008E827525
:100B8300830012074A60060EEE656270F0C2D5EB71
:100B9300C0E0EAC0E0E9C0E0EE120DE9D0E0F9D030
:100BA300E0FAD0E0FB120731FF60AAEBC0E0EAC035
:100BB300E0E9C0E0120A8BD0E02401F9D0E0340070
:100BC300FAD0E0FBE5620460DCD562D98087D22AE3
:100BD30080A2120DCC60F7E562700104120509A929
:100BE30062600DE562600914F562120E73EF60F343
:100BF300EA30E702F404C3995077EAF4256204303B
:100C0300E701E404F562800D120DCC60C1EA0562D0
:100C13002562120509EA785FF630E701E4256204EC
:100C2300D56204202D0114120DE9E4C0E0120E7305
:100C3300785FE6601320E70714F6120A7380220434
:100C4300F6D0E014C0E07F00120A73E56260071279
:100C53000A6A1562800B302D03120A6AD0E0020A79
:100C6300C4D0E00480C5120DCC60A0E56204120577
:100C730009785FEAF6E562202D026001042404127C
:100C83000DE974FF04C0E0120E73120A73E56220CB
:100C93002D026003120A6AD0E0B562E87F45120AAA
:100CA3007D785FE67F2B30E7047F2DF404C0E012EC
:100CB3000A8BD0E075F00A84C0F0120A74D0E012F7
:100CC3000A74020AC4791080027908C22EC23080E5
:100CD30008D2D5790A8004790AC2D5E56204700284
:100CE300F562E4FAFDFEFF120A50FC7B082029138B
:100CF300120A50FD7B1030280A120A50FE120A50C5
:100D0300FF7B20EC3382D592D55013C3E430280601
:100D13009FFFE49EFEE42029039DFDE49CFCE4CBBD
:100D2300F8C229EC700CCFCECDCCE824F8F870F3E0
:100D33008017C3EF33FFEE33FEED33FDEC33FCEBF3
:100D430033FB994002FB0FD8E9EB302905F8D0E0DB
:100D5300C448B229C0E00AEC4D4E4F78207B0070A6
:100D6300C2EAB5620040BCC0E0120DEBD0F0D0E0A7
:100D7300202904C4C0E0C4B229C0F0120A74D0F020
:100D8300D5F0EB020AC41209F80B61530CC8580BD7
:100D9300324C0B2E420CCC4F0CD4440CD4490B4791
:100DA300430CDA550C0B460C69450BD5470EA05086
:100DB3000B362D0B3A2E0B5D2B0B3E230B5B200EBC
:100DC300892A0AF64800000B55E562B4FF037562F1
:100DD30006120A50FC120A50FD120A50FE120A5063
:100DE300FF7858020538790AA2D5202B14302D0933
:100DF300B910020404B9080104A2D5202E0250013F
:100E030004202A68922AB561005034C0E07F203064
:100E13002B197F30A22A722E722D500F120E42C24E
:100E23002AC22EC22DC2307F30800F302D03E9C07D
:100E3300E0120A8B302D03D0E0F9D0E0B561CC305D
:100E43002D177F30B9100C120A8B7F58302C077F77
:100E5300788003B90803120A8B302A057F2D020A12
:100E63008B7F202030F87F2B202EF322922A80CFF5
:100E73007F00B4070050052458F8E6FF22286E755A
:100E83006C6C2900D229120A503029F8C2297861E2
:100E930030D50108F6020AF62D50434958120A507C
:100EA3002403B405004001E4900E9B93120A7C7462
:100EB3003A120A7CD22B756104020CC825730020F8
:100EC3002573003E005F2573002020202020202072
:100ED3002020202020202020004B4D480025337562
:100EE300004D5048003C005F257320202020202027
:100EF300202020202020002530337520004C415431
:100F03005F3A5F25635F25303375405F2530322EAE
:100F13003032662720004C4F4E5F3A5F25635F25D2
:100F2300303375405F2530322E303266272000443F
:100F330049525F3A5F2530337540002533627500AF
:100F43005E0025733A2025362E3166204D69002533
:100F5300733A2025362E3166204B4D0025733A20F7
:100F6300252D322E316600560025733A20256278EE
:100F73002E253162780025733A20002562752F25CE
:100F830062752F25347500204B204D204820284BB7
:100F93004D2F482900204D2050204820284D494CF2
:100FA300452F482900474D5420202B2562642000FB
:100FB300474D54202025626420200025735F25734C
:100FC3000053654C454354494F4E5F44274D4F44AE
:100FD3004520004C494D4954452020202020202005
:100FE3002020202000504F494E545F5554494C490E
:100FF3005341542E20200065434C414952414745FB
:101003002020202020202020005265474C414745C6
:10101300535F44555F504159532000494E464F5F3B
:1010230044555F535953547A4D4520200020554E63
:101033004954652020202020202020202000204605
:1010430055534541555F484F524149524520002071
:10105300534F4E5F44455F434C4F43484520200068
:10106300FF6393FF6515FF585BFF7115FF6221FF57
:101073003C68FF6471FF71E3FF66A6012200012053
:10108300000123000121004188100044880600006C
:101093000000418811004188040041880F00418805
:1010A3000D004188050041880200418621004185E9
:1010B3001F0041852000448737000000004A874D08
:1010C300000000000000000000004A874300000009
:1010D3000000000000000044872D0000000042874C
:1010E3002B00004487330000000041873100418713
:1010F3005D0042872000004187320042875B1C204D
:10110300448722000000004187290041872A0041CB
:1011130087280044875E0000000041876300418701
:101123006400418762004487570000000044871C25
:101133000000000044873F00000000418726004173
:101143008727004A87920000000000000000FF008C
:101153004A879C0000000000000000FF004287A6B1
:1011630000004287B600004E87A800000000000080
:1011730000000000000000004187B9004187B8006B
:101183004A88230000000000000000FF0042882D71
:1011930000004A882F0000000000000000FF00420A
:1011A300883900004987C7000502010504020506C6
:1011B3004987BE0005020105040205064187D100E7
:1011C3004187D0004287D200004187D4005687D799
:1011D30000000000560000000000000000000000B6
:1011E30000FF0000000002A4862202A686224C878C
:1011F300F51F1C1F1E1F1E1F1F1E1F1E1F41841BAA
:101203000002A8000041883B0041883CFF01AA007E
:1012130041883D0041883F0041883E000124000091
:1012230025730025336275005E004E452533750036
:101233004520253375005345253375005320253349
:10124300752A00534F253375004F20253375004E03
:101253004F253375004E202533750025336C7500FB
:101263004D00202020203E002020203E3E00202054
:101273003E3E3E00203E3E3E3E003E3E3E3E3E0063
:1012830025732020200025733E20200025733E3E39
:10129300200025733E3E3E00253475004D50480026
:1012A3004B4D48004E452533754000452025337589
:1012B30040005345253375400053202533754000C6
:1012C300534F25337540004F2025337540004E4F53
:1012D30025337540004E2025337540002020202003
:1012E30020400025352E3166204D690025352E31ED
:1012F30066204B4D00253262753A25303262750007
:101303002573253262753A2530326275007E0025D9
:10131300362E3166204D690025362E3166204B4D21
:1013230000253375204D504800253375204B4D481B
:101333000025342E3166204D50480025342E316669
:10134300204B4D4800253262752F253262750025EA
:10135300733A252D322E316656004241540025350D
:101363002E31664D690025352E31664B4D002533F0
:10137300754D5048002533754B4D48002533750096
:1013830044495F2573002532750025735F4445008A
:101393005175696E74657A7A00414C4552544552D1
:1013A30000475053202573002573202573202120E7
:1013B30020003A70FA83BCAAE9E43E81E0F8BF9DBD
:1013C300E9E63F80000039283C1ABB9969663DA3D2
:1013D30035E3BF255DE73FC90FDB418DDBCCC44956
:1013E30036EE45C9913FC5B0F83D3F800000C317B5
:1013F300F534452FFA73C60AFDDD1214A404A2E1E5
:1014030092281420E0159013B5740412044C80261E
:101413001214A430E102B22820E0EB8C278D288E31
:10142300298F2A9013C9740412044CA827A928AA47
:1014330029AB2A120169ED4C6007302804EC648063
:10144300FC221214A4C0E08C278D288E298F2A90A9
:1014530013ED740312044CA827A928AA29AB2A1256
:101463000169ECC527FCEDC528FDEEC529FEEFC5D6
:101473002AFF9013DD740312044CD082A827A928F5
:10148300AA29AB2AE58230E007120272B22880A6AD
:10149300EFCBFFEECAFEEDC9FDECC8FC1202728071
:1014A30095ED33EC547FCC33922824605007D0E081
:1014B300D0E00204377B837AF97922783E120169FE
:1014C300EDF933ECF83324815011EFFBEEFA1203FC
:1014D300CB12038DECB2E7FC120078ED33EC3360F2
:1014E3002F2403F8C313FCED92E7FDE82481E450B5
:1014F3001FECF8EDF9EEFAEFFB1203CBEF04C2E0B9
:10150300FCF582120397ECB2E7FC120078E5820344
:10151300FAED33EC3360071413FCED92E7FDEA2296
:10152300BE1249253E4CCCCDBEAAAAAB3F800000DB
:101533003E7ADBB03EED63383F24BC7D3F490FDB91
:10154300ED33ECC2E7CC339228B4FF13ED547F6044
:10155300030204377FDB7E0F7DC97C3F02163EC248
:1015630029C3947F401E7007EDD2E794904015EF96
:10157300FBEEFAEDF9ECF87F007E007D807C3F12F4
:101583000272D229ED33EC33248430E705E4C0E062
:10159300806D04FAEDD2E754F0C333DAFD54073417
:1015A300002323C0E0CCC0E0F8EDC0E0F9EEC0E0DA
:1015B300FAEFC0E0FBE4120397EC24FEFC8C388DB9
:1015C300398E3A8F3B1201697B007A007980783F2C
:1015D300120078ECC538B2E7FCEDC539FDEEC53A2B
:1015E300FEEFC53BFFD0E0FBD0E0FAD0E0F9D0E05E
:1015F300F8120078A838A939AA3AAB3B1202728CC8
:10160300388D398E3A8F3B901523740312044CA8FE
:1016130038A939AA3AAB3B120169D0E0600F242FF5
:10162300F582E43415F5831209B412007830290BDE
:101633007BDB7A0F79C978BF120078ED33EC336026
:1016430006ECA22892E7FC22C229C22AC22BC22C92
:10165300F9E4F52EF52FFCFDFEFFE91028EA202B17
:101663000CB42D04D22BD322B42B02D32224D0507A
:101673004794095041240A302C15F8852FF0740A39
:10168300A42872E74051C5F0704D85F02FD322D2C4
:101693002AC0E0E4FBFA79207841120169ECF8ED05
:1016A300F9EEFAEFFBD0E0FCE41203971200783076
:1016B30029B4152ED322240A202C20B4FE07202976
:1016C3001AD229D32224EB600424E0700EA22B92B9
:1016D30029D22CC22BD322C3020437E4302C0BE5CE
:1016E3002F302B02F404A229922B302AEA252E2034
:1016F300D2E5A2E7922C5002F404B4260050D8CCD1
:10170300C0E0EDC0E0EEC0E0EFC0E0EC1204C9D0F1
:10171300E0FFD0E0FED0E0FDD0E0FC202C0512017C
:10172300698003120272302B0312037CC32202046A
:101733003722EDA2E7D2E7F9EC3340F260F3B4FFCE
:1017430008ED547F70E8020441F82481C2E0C0E050
:10175300F40428FAC313FCED92E7FD8C308D318E2F
:10176300328F33EEA2E7E9BA7F02C3133400940049
:10177300FA75F091A4E5F013F494FE8AF0A433E52E
:10178300F033248CD313FDE492E7FE7F007C3F7596
:101793008302ECC0E0F8EDC0E0F9EEC0E0FAEFC080
:1017A300E0FBAC30AD31AE32AF33120272D0E0FBAE
:1017B300D0E0FAD0E0F9D0E0F8120078ED6480FDD3
:1017C30030E7011CD583CBED33CC33F8D0E0A2E76F
:1017D3001328C313CC13FD227581AA02181C0231EE
:1017E3001FE493A3F8E493A34003F68001F208DF18
:1017F300F48029E493A3F85407240CC8C333C454D6
:101803000F4420C8834004F456800146F6DFE48089
:101813000B010204081020408090107EE47E0193A7
:1018230060BCA3FF543F30E509541FFEE493A3605B
:10183300010ECF54C025E060A840B8E493A3FAE4B6
:1018430093A3F8E493A3C8C582C8CAC583CAF0A307
:10185300C8C582C8CAC583CADFE9DEE780BE8F3345
:101863008E328D318C30AB37AA36A935A8341202AB
:10187300721215438F338E328D318C30E53430E75D
:1018830047ECC0E0EDC0E0EEC0E0EFC0E0E4FFFEF7
:10189300FDFCAB33AA32A931A83012030F7BDB6006
:1018A3000250087A0F7949784080067A0F7949788F
:1018B300C0D0E0FFD0E0FED0E0FDD0E0FC12007825
:1018C3008F338E328D318C30AF33AE32AD31AC309D
:1018D300228B278A288929AB2AAA2BA92C12073104
:1018E300FEAB27AA28A929120731FF6E702BEF60E0
:1018F3000DE52E152E7002152D14452D70037F0056
:101903002274012529F529E43528F5287401252CAD
:10191300F52CE4352BF52B80BEAB27AA28A9291279
:101923000731FFD3EE6480F8EF64809840037F01B2
:10193300227FFF22D2288B2B8A2C892D121973C068
:10194300E0FF121A12D0E040F312165E400122ECBF
:10195300C0E0EDC0E0EEC0E0EFC0E0121973D0F0DC
:10196300AFF0D0F0AEF0D0F0ADF0D0F0ACF080D965
:10197300E475F001782B1209E8020731257300534F
:1019830050454544005253002533754D50480025BA
:1019930033754B4D48004C41534552003E3E3E008B
:1019A3004B412042414E4400256264004B2042419A
:1019B3004E4400582042414E440085434C85444DDB
:1019C30085454EEBC546FBEAC547FAE9C548F97FAD
:1019D30009784F120731F60809E970010ADFF4AB01
:1019E30046AA47A948020AACEFB40A07740D1219B4
:1019F300F6740A309811A899B8130CC2983098FD60
:101A0300A899C298B811F63099FDC299F59922EFB9
:101A1300C394094005EF940E4003BF2003D3800114
:101A2300C3222533750025730025733100257332D6
:101A33000025730025733A2575005F564F4C554DAD
:101A43004520202020202020202000434F4E4E45BB
:101A5300435445525F4750530056495445535345E9
:101A630000414C41524D4500414C4C554D6500657C
:101A73005445494E540043414D6552410042494447
:101A830049524543542E00444520524F5554450076
:101A9300434F4E54524F4C450046494E2044450057
:101AA30044414E47455245555800504F494E540006
:101AB30041564552544953532E005554494C4953AA
:101AC30041542E005F504F494E5400414A4F5554E4
:101AD3006500504C45494E005355505052494D6591
:101AE3000056494445004D454E555F5052494E43BB
:101AF3004950414C0053654C454354494F4E5F4454
:101B0300555F4D4F4445004C494D495445005F6571
:101B1300434C41495241474520202020202020208A
:101B2300005265474C414745535F44555F50415907
:101B3300532000494E464F5F44555F535953547ADF
:101B43004D45202020005553455220494E464F0015
:101B53005F554E495465202020202020202020203E
:101B6300200046555345415520484F52414952455F
:101B730000534F4E00534F4E20444520434C4F4398
:101B830048450052454D495345005452414A455436
:101B9300004465464155540044655441494C530043
:101BA300434F4E464F5254004F5549004E4F4E003F
:101BB300424F5553534F4C45004F444F00444154FB
:101BC3004500546563686E6F6C6F676965004155C6
:101BD300544F2D5445535400415543554E455320BE
:101BE300444F4E4E45455300545249502054494D9D
:101BF3004500424154544552494500534F465457BA
:101C030041524500444F4E4E4545532000534155E4
:101C13005645474152446500504F494E5453204462
:101C2300275554494C492E00522F4F444F004D4FD6
:101C330059454E00484555522E0000000000000053
:101C430000004F4F000000060006000000487A41E4
:101C53000000F8252524F800007F25251A007D4182
:101C630040417D000000000B070000487A49000056
:101C7300F824252525F803030000000008083E0882
:101C83000800000000583800080808080800000091
:101C9300400000002010080402003E5149453E0068
:101CA30000427F40000042615149460022414949B8
:101CB30036001814127F10002745454539003C4A69
:101CC3004949300001710905030036494949360085
:101CD300064949291E00003636000000005B3B0020
:101CE300000000081C3E7F001414141414007F3EEF
:101CF3001C080000020159090600324959413E00FF
:101D03007E1111117E00417F494936003E41414118
:101D13002200417F41413E007F49494141007F0903
:101D2300090901003E4149497A007F0808087F00FC
:101D330000417F4100002040413F01007F08142201
:101D430041007F40404040007F020C027F007F0241
:101D530004087F003E4141413E007F090909060016
:101D63003E4151215E007F09192946002649494910
:101D7300320001017F0101003F4040403F0007184E
:101D8300601807003F4038403F00631408146300A5
:101D9300070870080700615149454300007F41412E
:101DA30000000204081020000041417F00000402EB
:101DB30001020400404040404000000402010000D2
:101DC3002054545478007F484444380038444444F1
:101DD3002000384444487F00385454540800087E97
:101DE30009020000081454543C007F0804047800DE
:101DF30000447D4000002040443D0000007F102847
:101E0300440000417F4000007804180478007C08F7
:101E1300040478003844444438007C142424180013
:101E23001824147C4000007C0804040048545454D3
:101E33002000043E442000003C4040207C001C2045
:101E430040201C003C4030403C0044281028440003
:101E53004C5050503C004464544C440000083641FC
:101E6300000000007700000000413608000008046D
:101E7300081008002A552A552A000800000000000F
:101E830000000000000000000000000400F8F8005B
:101E9300000D0D000638380038380000000000003F
:101EA300000820F8F820F8F82000020F0F020F0FA7
:101EB3000200003078CE8E18100000040C38390F61
:101EC300060008183C24BCD86030000006030E1E30
:101ED300121E0C0800B0F8487830000000070F0805
:101EE30009070F09023838000004E0F81C04030F47
:101EF3001C1004041CF8E0101C0F030780A0E0C0B2
:101F0300E0A08000020301030200068080E0E0807D
:101F130080000003030000030000002C3C1C06802B
:101F2300808080808000000000000004000000002A
:101F3300000C0C00060000C0F03C0C0C0F0300006A
:101F4300000800F0F80868F8F00000070F0B080F0E
:101F530007000800202030F8F80000000000000F00
:101F63000F0000080030380888F87000000C0E0BD2
:101F730009080800080030388888F8700000060E49
:101F830008080F0700080000F8F800E0E00000036D
:101F93000302020F0F020800F8F88888880800007F
:101FA3000808080C0703000800C0E07858C8800040
:101FB30000070F08080F07000800080888E87818CA
:101FC3000000000E0F01000000080070F8C888F838
:101FD300700000070F08090F07000800F0F8080851
:101FE300F8F0000000090D0F030100080000006075
:101FF300600000000000000C0C000000080000005E
:1020030060600000000000002C1C0000000700803E
:10201300C0E0F0F80000000103070F0005606060F6
:1020230060000C0C0C0C000700F8F0E0C08000000E
:102033000F07030100000760701090F060000000BC
:102043001B1B0000000400382838000000000800B3
:10205300E0F01818F0E000000F0F01010F0F000867
:1020630000F8F88888F87000000F0F08080F0700C1
:102073000800F0F8080838300000070F08080E06BB
:10208300000800F8F80818F0E000000F0F080C072C
:1020930003000800F8F88888880800000F0F080874
:1020A3000808000800F8F88888880800000F0F0067
:1020B300000000000800F0F8080838300000070F9F
:1020C30008090F0F000800F8F88080F8F800000FE7
:1020D3000F00000F0F0008000008F8F808000000C8
:1020E30000080F0F080000080000000000F8F800C7
:1020F30000060E08080F07000800F8F880E07818BB
:1021030000000F0F00030F0C000800F8F800000098
:102113000000000F0F08080808000800F8F820C0A6
:1021230020F8F8000F0F0001000F0F0800F8F86007
:10213300C080F8F8000F0F0000010F0F0800F0F83F
:102143000808F8F00000070F08080F07000800F858
:10215300F88888F87000000F0F00000000000800E6
:10216300F0F80808F8F00000070F08181F17000818
:1021730000F8F88888F87000000F0F00010F0E00B8
:1021830008003078C88818100000040C08090F06EE
:102193000008000808F8F80808000000000F0F0006
:1021A30000000800F8F80000F8F80000070F08081E
:1021B3000F07000800F8F80000F8F8000003070C08
:1021C3000C0703000800F8F800C000F8F800010F3E
:1021D3000E010E0F0108001838E0C0381800000E79
:1021E3000F00010F0E00080078F88080F8780000D7
:1021F30000000F0F0000000800080888C8783800A6
:10220300000E0F09080808000404FCFC00101F1F3F
:10221300000638F8C00000000000030F0C0004FCA7
:10222300FC04001F1F1000080C1E92DE6C30180007
:10223300000301060F090F06040000000000000060
:10224300000400000000000000000800F2FA181863
:10225300FAF200000F0F01010F0F000800FAFA0055
:1022630000FAFA0000070F0C0C0F07000800F2FA3F
:102273000808FAF20000070F08080F07000800F02B
:10228300FA1A19F9F000000F0F01010F0F000800EF
:10229300F8FA8A89890800000F0F0808080800085F
:1022A30000080AFAF90908000008080F0F080800D7
:1022B3000800F0FA0A09F9F00000070F08080F07F1
:1022C300000800F8FA0201F9F80000070F08080FE8
:1022D30007000800FAF9C382F9F800000F0F0001A4
:1022E3000F0F000800F8FA0101FAF80000070F0CBD
:1022F3000C0F07000800F8F9898A8A0800000F0FFD
:10230300080808080008000809F9FA0A0800000884
:10231300080F0F0808000800F0F9898AFAF0000096
:102323000F0F01010F0F000800F8044444788000E8
:10233300000F0002020201000800C0E02020E0C0FC
:102343000000070F08080F07000800E0E02020E066
:10235300C000003F3F08080F07000800C0E020202E
:10236300E0E00000070F08083F3F000800E0E080BE
:1023730040606000000F0F00000000000800C0E094
:10238300202020200000080909090F06000800206A
:10239300F8F8202020000000070F080808000800B4
:1023A300E0E00000E0E00000070F08080F0F00085E
:1023B30000E0E00000E0E0000003070C0C0703006E
:1023C3000800E0E000C000E0E000030F0C030C0F86
:1023D30003080060E08080E06000000C0E03030E41
:1023E3000C000800E0E00000E0E000002327341CBC
:1023F3000F03000800F9F98A8A8A0800000F0F0802
:1024030008080800FF1E7DFF1E8EFF1E97FF1EA4F7
:10241300FF1EB5FF1EC5FF1ED6FF1EE7FF1EECFF06
:102423001EF5FF1EFEFF1F0DFF1F1AFF1F21FF1FBB
:102433002EFF1F37FF1F44FF1F55FF1F66FF1F7728
:10244300FF1F88FF1F99FF1FAAFF1FBBFF1FCCFFA2
:102453001FDDFF1FEEFF1FFFFF2010FF201FFF20C8
:102463002AFF2039FF2048FF2051FF2062FF2073FD
:10247300FF2084FF2095FF20A6FF20B7FF20C8FF81
:1024830020D9FF20EAFF20FBFF210CFF211DFF21A4
:102493002EFF213FFF2150FF2161FF2172FF218386
:1024A300FF2194FF21A5FF21B6FF21C7FF21D8FFFC
:1024B30021E9FF21FAFF220BFF2214FF2221FF2231
:1024C3002AFF223BFF2244FF224DFF225EFF226FA1
:1024D300FF2280FF2291FF22A2FF22B3FF22C4FF2B
:1024E30022D5FF22E6FF22F7FF2308FF2319FF234C
:1024F3002AFF233BFF234CFF235DFF236EFF237F34
:10250300FF2390FF23A1FF23B2FF23C3FF23D4FFA5
:1025130023E5FF23F60CF0F8FCFEFE0E8EFEFEFC18
:10252300F8F0FFFFFFFFFFF81FFFFFFFFFFF0F1F85
:102533003F7F7F70707F7F3F1F0F0C0000707070B4
:1025430078FCFCFEFEFE00000000000000FFFFFF21
:10255300FFFF000000000000007F7F7F7F7F000CF3
:1025630000F0FCFCFE0E0EFEFEFCF8F00000008006
:10257300E0F8FEFFFF3F1F0300787E7F7F7F7F73BE
:10258300707070000CF0FCFCFEFE0E0EFEFEFCFCF8
:10259300F0C1C1C1C1DD1C3CFFFFFFF7E30F3F3FAB
:1025A3007F7F70707F7F3F3F0F0C000080F0FE3E07
:1025B300FEFEFEFE0000E0FCFFDFC3C0FFFFFFFFE7
:1025C300C0C00707070707077F7F7F7F07070CFE4A
:1025D300FEFEFEFE0E8E8E8E8E0E0E8F8F8F8F8FD3
:1025E3000303FFFFFFFFFE0F3F3F7F7F70707F7F7F
:1025F3003F3F0F0CF0F8FCFEFE0E0E7E7E7C7C70DF
:10260300FFFFFFFFFF0607FFFFFFFEFC0F3F3F7FBC
:102613007F70707F7F3F3F0F0C001E1E1E1E1E1E0D
:10262300FEFEFEFEFE00000000E0F8FFFFFF1F07B6
:10263300000060787F7F7F1F07000000000CF0FC24
:10264300FCFEFE0E0EFEFEFCFCF0E3F7FFFFFF1C9C
:102653001CFFFFFFF7E30F3F3F7F7F70707F7F3FDC
:102663003F0F0CF0FCFCFEFE0E0EFEFEFCF8F03FEE
:102673007FFFFFFFE060FFFFFFFFFF0E3E3E7E7E1A
:1026830070707F7F3F1F0F02707000000E0E020CF0
:10269300040CFEFEFCF8F0E0C08000000000FFFF29
:1026A300FFFFFFFFFFFFFF7E3C187F7F3F1F0F07EA
:1026B3000301000000000E040C1E1E0C00000000AD
:1026C300000000000E00C0FEFEFEFE1EFEFEFEFE2B
:1026D300C00000E0FFFFFFFF878087FFFFFFFFE0F1
:1026E300007F7F7F7F07070707077F7F7F7F000CC0
:1026F300FEFEFEFEFE1E1EFEFEFCFCF0FFFFFFFFC5
:10270300FF1E1EFFFFFBFBF17F7F7F7F7F78787FBC
:102713007F7F3F1F0D0CFEFEFEFEFE1E1EFEFEFC17
:10272300FCF8FFFFFFFFFF0000FFFFFFFFFF7F7FBE
:102733007F7F7F78787F7F7F3F1F0BFEFEFEFEFE4D
:102743001E1E1E1E1E1EFFFFFFFFFF3C3C3C3C3CAB
:10275300007F7F7F7F7F7878787878780B0C0D0502
:10276300080DFEFEFEFEFE00C0F8FEFEFE3E06FF66
:10277300FFFFFFFF7FFFFFFFF78000007F7F7F7F6B
:102783007F00030F7F7F7F7C700AFEFEFEFEFE004C
:1027930000000000FFFFFFFFFF00000000007F7F3D
:1027A3007F7F7F7878787878110CFEFEFEFEF880C4
:1027B30000FEFEFEFEFEFFFFFFFFFF1FF8FFFFFF11
:1027C300FFFF7F7F7F7F7F00011F7F7F7F7F0CF075
:1027D300F8FCFEFE1E1EFEFEFCF8F0FFFFFFFFFFEF
:1027E3000000FFFFFFFFFF0F1F3F7F7F78787F7F92
:1027F3003F1F0F0C0C0CFEFEFEFEFE1E1EFEFEFE19
:10280300FCF8FFFFFFFFFF1E1EFFFFFFF7E37F7FC5
:102813007F7F7F00007F7F7F7F7F0DF0FCFCFEFECC
:102823001E1EFEFEFCFCF80083878F9F9F3F7F7E6A
:10283300FCF8F8F0C00F1F3F7F7F7878787F7F3FE9
:102843003F0F0C1E1E1EFEFEFEFEFEFE1E1E1E0083
:102853000000FFFFFFFFFFFF0000000000007F7F7D
:102863007F7F7F7F0000000C0F151EFEFEFEFEC063
:102873000000FEFEFEFEFE0000C0FEFEFEFE1E0089
:102883001FFFFFFFFF00FFFFFF03FFFFFF00FFFF2F
:10289300FFFF1F0000001F7F7F7F7E7F7F010001FE
:1028A3007F7F7C7F7F7F1F00000D063EFEFEF8E0EA
:1028B30000C0F8FEFE3E060000C0FFFFFF3FFFFF23
:1028C300FFC00000707E7F7F1F0100011F7F7F7E9E
:1028D300700D0A001E1E1EDEFEFEFEFE7E0080F050
:1028E300FEFFFFFF1F0300787F7F7F7F7F7878786D
:1028F30078FF2518FF253DFF2562FF2587FF25ACBF
:10290300FF25D1FF25F6FF261BFF2640FF2665FF87
:10291300268AFF2691FF2692FF2693FF2694FF2601
:10292300B9FF26BAFF26C7FF26F2FF2717FF27188E
:10293300FF273DFF275FFF2760FF2761FF2762FF18
:102943002763FF2764FF278CFF27ABFF27ACFF27F5
:10295300D1FF27F6FF27F7FF27F8FF281DFF28459C
:10296300FF286AFF286BFF286CFF28ACFF28D4FFE1
:1029730028D50B013C24242424242424243C000BA8
:10298300013C3C3C3C3C3C3C3C3C3C000A0200FEE1
:10299300020202020202FE00007F4040404040402B
:1029A3007F000A0200FEFEFEFEFEFEFEFE00007F2A
:1029B3007F7F7F7F7F7F7F00100200000000C0F0D9
:1029C300FC1E1EFCF0C000000000C0F0FCFFFFFF77
:1029D300FFC8C8FFFFFFFFFCF0C01E04000000009B
:1029E30000C0C00000181800001F0204081F0000E8
:1029F30018180000C0C0000000008040404C8C004C
:102A030000000000000000000000000000000000C3
:102A130000000000CC4C4040030404646300000049
:102A230000000000000000000000000000000000A3
:102A33000000676505050000000000000606003081
:102A4300300000B8A8A8E8000030300000060600F7
:102A530000000000100200000080E0F8FEFFFEF816
:102A6300E0800000000060783E3F1F1F0F0F0F1F24
:102A73001F3F3E7860001002030F3EFEFCFCF8F897
:102A8300F0F0E0E0C0C0800060783E3F1F1F0F0FF2
:102A930007070303010100001002030F3EFEFCFCC5
:102AA300F8F8F8FCFCFE3E0F030000000000030FE3
:102AB3003F7F3F0F030000000000100280C0C0E012
:102AC300E0F0F0F8F8FCFCFE3E0F03000001010308
:102AD3000307070F0F1F1F3F3E786000100200001F
:102AE3008080C0C0F0FCFFFFFCF080000000030307
:102AF30007070F0F0F1F1F1F3F3F7F7C70801002C0
:102B0300C0C0E0E0F0F0F0F8F8F8FCFCFE3E0E0187
:102B13000000010103030F3FFFFF3F0F010000000F
:102B23001002010E3EFEFCFCF8F8F8F0F0F0E0E0D5
:102B3300C0C0000000010F3FFFFF3F0F030301016F
:102B43000000100200000080F0FCFFFFFCF0C0C09A
:102B53008080000000707C7F3F3F1F1F1F0F0F0FFF
:102B630007070303200400000000000000000080AA
:102B7300C0E0F0F8FCFEFCF8F0E0C08000000000CC
:102B83000000000000000080C0E0F0F8FC1E1FFF02
:102B93000FFF03132B13030303030303FFFEFCF8CD
:102BA300F0E0C080000000000103070F1F3C7CF130
:102BB300F0F7E0E0E0E0E0E6E9E9E6E07F3F1F0F61
:102BC30007030100000000000000000000000000F7
:102BD3000103070F1F3F1F0F070301000000000041
:102BE30000000000000020040000000000000000BE
:102BF3000080C0E0F0F8FCFEFCF8F0E0C0800000CC
:102C030000000000000000000080C0E0F0F8FC1E9F
:102C13001F0FFF03132B13030303030303FF0F1EF2
:102C23001CF8F0E0C080000000000103070F1F3C08
:102C33007CF0F7E0E0E0E0E0E6E9E9E6E0F7703CAD
:102C43001C0F07030100000000000000000000004B
:102C530000000103070F1F3F1F0F070301000000C0
:102C6300000000000000000020040000000000003D
:102C730000000000000000C0F0F8F8F0C000000001
:102C83000000000000000000000000000000000041
:102C9300000000C0F0FCFFFF03030303FFFFFCF091
:102CA300C00000000000000000000000000000C0A1
:102CB300F0FCFFFFFFFFFFFF60606060FFFFFFFFAF
:102CC300FFFFFCF0C0000000000000000000070F41
:102CD3000F0F0F0F0F0F0F0F0C0C0C0C0F0F0F0F0D
:102CE3000F0F0F0F0F07000000001803FC02010174
:102CF30001010181C1E1F1F9F9F1E1C181010101B1
:102D0300010102FCFF0000000406070707FFFFFFA5
:102D1300FFFFFF0707070604000000FF3F40808016
:102D230080808080809F9F9F9F9F9F8080808080E6
:102D33008080403F1803FC02010101E1E1E1E1E190
:102D4300E1E1E1E1E16121010101010102FCFF0097
:102D5300000000FFFF7F3F3F7FFFFFFFFCF8F0E035
:102D6300C080000000FF3F408080808180808080A1
:102D730080808183878F8F8783818080403F180382
:102D8300FC02010101010181C1E1F1010101010124
:102D930001010101010102FCFF0000183C7EFFFF5D
:102DA300FFFFFF7E7E7E7E7E7E7E7E7E7E0000FF38
:102DB3003F4080808080808183878F808080808077
:102DC300808080808080403F1803FC020101010164
:102DD30001010101010101F1E1C1810101010101D0
:102DE30002FCFF00007E7E7E7E7E7E7E7E7E7EFFF8
:102DF300FFFFFFFF7E3C180000FF3F408080808084
:102E0300808080808080808F8783818080808080A5
:102E1300403F1803FC0201010101012161E1E1E1ED
:102E2300E1E1E1E1E1E1E101010102FCFF00000078
:102E330080C0E0F0F8FCFFFFFF7F3F3F7FFFFF0014
:102E4300000000FF3F4080808183878F8F878381CD
:102E530080808080808081808080403F07011C22A9
:102E6300514945221C30060000000000000080C0CC
:102E7300E0E0F0F8F8FC7C7E3E3E3E3E3F1F1F1F25
:102E83001F1E3E3E3E3E7C7CFCF8F8F0E0E0C08036
:102E9300000000000000000000C0F0F8FEFF7F3FCC
:102EA3000F07030101000000000000000000000004
:102EB300000000000080C0E0F0F9FDFF7F3F3F7F8E
:102EC300FFFEF8F0C00000E0FFFFFFFF3F0100003E
:102ED3000000000000000000000000000080C0E0CF
:102EE300F0F8FCFE7F3F1F0F070301000000000006
:102EF300013FFFFFFFFFE0037FFFFFFFF8800000BC
:102F0300000000000080C0E0F0F8FCFE7F3F1F0FD0
:102F130007030100000000000000000000000000A3
:102F230080F8FFFFFF7F030000030F1F7FFFFEFCFE
:102F3300F0F8FCFEFF3F1F0F070301000000000035
:102F43000000000000000000008080C0E0F0FCFEF4
:102F5300FF7F1F0F030000000000000000000103BB
:102F630007070F1F1F3F3E7E7C7C7C7CFCF8F8F834
:102F7300F8787C7C7C7C3E3E3F1F1F0F07070301D4
:102F83000000000000000010010000007C92107C93
:102F93004444447C10927C000020040000000000A4
:102FA3000000000000000000FCE2820202040408AA
:102FB3000810A040A0100806060000000000000052
:102FC3000000000000000000FFFFFFFEFCF8F8E433
:102FD300C28100000001020C30C0000000000000AC
:102FE3000000000078FCFEFFFFFFCF8707070707FD
:102FF3000707070706060404040300000000183C43
:103003003C3C3C3C3C3C3D3F3F3F3F3F3F3E3C3CE8
:103013003C3C3C3C3C3C3C180000001201100100CD
:1030230000000883040000000101020001090921D6
:1030330000010001222E0009022200010100C0FA52
:10304300090400000103000000092100010001221E
:103053002E000705810308006400002E06A0FF0967
:10306300A5A10109A609A51580257F75089540B17D
:103073000209A71580257F75089508810209A915FE
:1030830080257F750895409102C0040309041A0343
:10309300570049004C004C002000540052004E00E1
:1030A3004900430053000000180347005000530039
:1030B300200041004C0045005200540045005200DE
:1030C300FF308DFF3091FF30AB0099A3ADB8C2CC78
:1030D300D6E0EBF500919293949597999B9EDE0031
:1030E3000000000000000000000000000000123B90
:1030F3003C1242DBF17812608B1247FA12679F127F
:103103006E20E4F522F523F521F5249087B9F0D25A
:103113000C90880D04F012487002002611F112562B
:1031230090124A59EF640A706A124B02EF60482406
:10313300FA7060123EFBD11B9087A6E07002A3E0F9
:103143007002B129900013E054FDF0A20DB3920D6B
:1031530090875BE07002A3E060031279D09087A6AA
:10316300E07002A3E0600890879BE0FF12571120F4
:103173001921125131801C900013E06402F0126E89
:10318300F8126F2931FD90875BE07002A3E06003C2
:103193001279D0124870300828201A25201B2220CB
:1031A3001C1F201D1C201E19201F16C39087E7E03B
:1031B300941E9087E6E0940040051276998002C23F
:1031C3002030081F20201C201A19201B16201C1336
:1031D300201D10201E0D201F0AF17890880BE0FFA0
:1031E3001251BC1243161260A4123BCD90841BE013
:1031F30070022124126D9A020033300802612B9071
:10320300875DE004F0E0D394034002E4F0F1787AC0
:103213002F7B9C752C037D047F0571547871766E2A
:103223007871E6FFD3947850157B017D039167781D
:1032330071E6FF7B3F7D07916778710680E27871C5
:1032430076037871E6FDD3940650157BFF7F6E916C
:10325300677871E6FD7BFF7F78916778710680E27E
:1032630090875DE07027752EFF752F12753083F1FF
:10327300DB915F7D037F28915D7D047F41915D7DBF
:10328300057F32915D7D067F4DB10B40E490875DF4
:10329300E064017029752EFF752F12753089F1DBFB
:1032A30091527D037F48915D7D047F37915D7D055C
:1032B3007F30915D7D067F3F7154B11740E2908767
:1032C3005DE064027027752EFF752F1275308FF144
:1032D300DB915F7D037F37915D7D047F4C915D7D45
:1032E300057F41915D7D067F52B10B40E490875D80
:1032F300E064037033752EFF752F12753095F1DB83
:1033030091527D037F2D915D7D047F4A915D7D0503
:103313007F43915D7D067F3671547871E6FF7BFFB5
:103323007D049167B10D40D822752F007530067565
:1033330031FF75321A7533C77B027D1E7F0112433D
:10334300817E887F23125E4F7A2C7B6BE4F52CFD04
:10335300FFF1FCF1F0E493787AF6F1F0740193084D
:10336300F6E47879F67979E7C3787B96400281268B
:10337300E47878F67878E6FFC3787A96400281217C
:10338300E52C701FE5282FFFE433FE18E6FD252901
:1033930012476A1278DEC083C082F1A3E493FFEC84
:1033A3004F8036E52C640170161279C112476A12F8
:1033B30078DEC083C082F1A3E493FFEC5F801AE55B
:1033C3002C6402701B1279C112476A1278DEC08323
:1033D300C082F1A3E493FFEC6FD082D083F08039F5
:1033E300787AE6FF18E6F98FF0A4F1F0A3A325821B
:1033F300F582E58335F0F58318E6FFF1C1E493FE2A
:10340300EFFDE5282DFDE433FCE5292912476A2D5C
:10341300F582E5833CF583EEF07878066177787979
:10342300066168E528787A26FFE5290826FD908459
:1034330000EFF0A3EDF0EFD3947F40069084007487
:103443007FF0EDD3940740069084017407F0227A4D
:103453002F7B8A752C037D027F5071547A2F7B8AD0
:10346300752C032275F080ED12476D2FF1C3E04BED
:10347300F022F178787376037873E6FFC3947D5076
:10348300157B017D0191677873E6FF7BE07D0691F3
:103493006778730680E2787376027873E6FDC394E7
:1034A3000650177BFFE4FFF1D27F7FF1D27F7EF1DD
:1034B300D27F7D916778730680E07BFF7D01E4FF17
:1034C30091677B3F7D06E4FF127B5C7F0191677B05
:1034D300607D067F01127B5C7F0291677BE07D0646
:1034E3007F0291677BFC7D017F7FF1CB7F7F9167BB
:1034F3007BFE7D017F7EF1CB7F7E91677BFF7D012C
:103503007F7DF1CB7F7D816771547871E6FF7BFF0F
:103513007D0591677871E6FF7BFF7D069167787182
:1035230006E6D39478221278D4F17890882DE0704F
:1035330002A3E0700C125A5C90882DEEF0A3EFF01A
:1035430022201B467A887B237D167FBC7E02D10511
:103553006031E4D10E602CD21B1278E7FF123FBA20
:10356300712C12562D90879BE0C4540F75F00AA45A
:10357300126FDC95F040077F097EB012563130B7E9
:103583004C80FBE4D10E70458040201C247A887B5C
:10359300237D167F2C7E01D105600FE4D10E600AD6
:1035A300D21C12562D12562D8023E4D10E701E808C
:1035B30019201A197A887B23B1FF6009E4D10E60C0
:1035C30004D21A8008E4D10E7003126F2990882D5B
:1035D300E07002A3E060167A887B23127986E4D137
:1035E3000E6007E47FFFD10F7003126F29301B0BAE
:1035F3001278E7123FB8712C124E70227D5A7F0F5A
:103603007E00D1F078711209C474FFFFFEFDFC78CF
:10361300711209A7C30209671278D49087B8E0FF33
:10362300A3E004F0C39F4002E4F0126E17FF9087FB
:10363300B9E0FE044F9000E0F0D2AFEE25E024A8FD
:10364300F582E43487F583E0FFA3E09087B6CFF0FB
:10365300A3EFF0F178125BFDEF4E6025D21DC21E81
:10366300C21F7E877F927C887D2F126CE112562DBC
:10367300124E6112431690879BE0FF126F5220B7E0
:10368300FD9087A6E07002A3E06061301D5E201EFE
:10369300297A877B927D167F2C7E01D1056014E405
:1036A300D10E600FD21E124E7090879BE0FF126FF7
:1036B300E88023E4D10E701E8019201F197A877BBE
:1036C30092B1FF6009E4D10E6004D21F8008E4D1F7
:1036D3000E7003126EF87A877B92127986E4D10E0C
:1036E3006004D10C7003126EF8124E61228E27F122
:1036F300FCE4FFFEFDFC127A04126977127A0412CD
:103703006A17788EA607E6FFF46053908837E0FBCC
:10371300AD29125B6AEF6043127ACAF583127A9875
:10372300500912478CED24B4FB800A127ACA12475F
:1037330086AF05AB07788EE6FFAD29125B6AEF60B3
:1037430017AE27AF28E4FCFD788A127A3A50057841
:103753008A02098B74FF8007E48004E48001E4FF9C
:10376300FEFDFC22F583E4740193FA740293F912CB
:103773000A1E120026E47876F6E47875F67875E684
:10378300FFD3947F500E08E612476A2FF1C3E4F08B
:10379300180680E9787606E6B408DEE4FDFF813199
:1037A300E0FC08E6FFED8FF0A4852B82852A83A336
:1037B300A32582F582E58335F0F5837878E62582C3
:1037C300F582E43583F5832291677BFF7D062291A1
:1037D300677873E6FD7BFF227531FF75321A753307
:1037E3004EFBFD7F011243817871766E22852B8219
:1037F300852A8322120026E1788F288D298A2A8B35
:103803002B22E4900005F0900003F090000774FF72
:10381300F0E4900009F09000137407F09000157421
:1038230002F090001714F09000B07438F09000B4D8
:103833007430F09000C77401F0228C6F8D70E4FE39
:10384300F9BF01051241468011BF020512413680BE
:1038530009BF0304F1F88002517D74A0F011AEEBAF
:10386300F053038011AE127AD4B503047E018005B0
:10387300BC20027901EE7003EC60E9E96401702871
:1038830011AEE05480B503027E01BF0105902555BA
:103893008013BF0205904555800BBF030590655506
:1038A300800390855574F0F0AF0622857082856F92
:1038B30083228F658B688A69896ACEECCECFEDCF80
:1038C3008E6D8F6EE56C156CAE6B7002156B4E6072
:1038D3002E12767C7002056914F9120731FBAD6E66
:1038E300AC6DAF65113D056EE56EAE6D7002056D95
:1038F30014F5828E83E0FF908461E02FF080C5226F
:1039030090849EE06002219490841CE024FD600278
:10391300219490849DE0FE7032EFD394014072EFC6
:1039230024FFFDE434FFFC908420E0FAA3E0FBC312
:103933009DEA9C5008CCEACCCDEBCD8004EF24FF6C
:10394300FD789EEDF6EE0408F6801BEFFDC3908430
:1039530021E09D31955005A3E0FF8000789EEFF6AE
:1039630090849DE008F690841D124123789FE624FD
:103973009EF9E43484FA7B0118E6756B00F56C114B
:10398300B5789E12785D700990841CF0A3E0FF5116
:103993006022908420E09400228F6590849CE060F4
:1039A30037E5656002415F90845C7405F090841C88
:1039B300E090845DF09000E0E090845EF09000E29F
:1039C300E090845FF078DF7C847D017B017A8479E9
:1039D3005C7E007F4002070B90841CE024FC705E39
:1039E300E5657020C3908421E0940731955005A3C9
:1039F300E0FF80027F07789EEFF6756501E490840F
:103A0300DFF08016C3908421E0940831955005A31C
:103A1300E0FF80027F08789EEFF690841EE0FEA30D
:103A2300E0FF74DF2565127B4D789EE6756B00F52C
:103A33006C12764B12785D702390841CF022E4782C
:103A43009FF6789FE6FFC394085011E5652F24DFA6
:103A5300F582E43484F583E4F00680E622BF0105B1
:103A63001241468011BF02051241368009BF03048B
:103A7300F1F88002517D74F0F02290855574AAF01C
:103A8300908AAA7455F09085552271E5AB207D008C
:103A93007C207F0151CB908803E0FB7D017C207F5C
:103AA3000151CB908812E0FB7D027C207F0151CB3A
:103AB30090880EE0FB7D037C207F0151CB90880B27
:103AC300E0FB7D047C207F018C298D2AE4FEF9BF75
:103AD30001051241468011BF02051241368009BF1C
:103AE3000304F1F88002517D74A0F0F1A4EBF053CC
:103AF3000380F1A4127AD4B503047E018005BC20AF
:103B0300027901EE7003EC60E9E964017028F1A425
:103B1300E05480B503027E01BF0105902555801353
:103B2300BF0205904555800BBF0305906555800383
:103B330090855574F0F0AF0622902000E0F5203018
:103B43000041E4908803F09088127405F090880E89
:103B53007409F0E490880AF090880BF090880C7454
:103B63000CF0C201C202C20012796C7D007C207F7E
:103B73000171E5F1EA518D127B3D51C7127B45512D
:103B8300C7D1D4902000E0F520A3E0908803F09003
:103B93002002E0908812F0902003E090880EF090CD
:103BA3002004E090880BF0902005E090880AF090C4
:103BB3002006E090880CF0783B7C877D017B017ABE
:103BC3006079007E007F0402070B3009147D007CBE
:103BD300207F01518D127B3D51C7127B4551C7C2D6
:103BE30009228C298D2AE4FEFDBF010A124146F108
:103BF300DC902AAA8020BF020A124136F1DC904AE7
:103C0300AA8013BF0309F1F8F1DC906AAA80075177
:103C13007DF1DC908AAA7455F0F1A47430F0F1A41C
:103C230012412CBB80047E018005BA20027D01EE87
:103C33007003EA60E9ED64017028AB04530380BBB1
:103C430080027E01BF01059025558013BF020590B8
:103C53004555800BBF0305906555800390855574CA
:103C6300F0F0AF0622E47872F6301102C1139084AB
:103C73001BE06002C11312377812669475321B750C
:103C83003336E4FB1258041264D7126E174401F062
:103C9300D2AF124870300119752EFF752F0F753092
:103CA30045127A8E1257AE90873BD12C1277FE8045
:103CB30014752EFF752F0F753052127A8E90873B35
:103CC300D12C124FCF126CD87B027D03E4FF124339
:103CD300817872E664017BFF7A1B79AB7028F1C1AE
:103CE300127A571243817BFF7A1B79AB1279EDFF6E
:103CF300C3743A9FFF752A017B3A7D03126006F174
:103D0300CF1279558022F1C1127A57F1BAF1D2124A
:103D130079557BFF7A1B79AF1279ED2443FB752A22
:103D2300017D037F43126006752EFF752F0F7530DB
:103D33005F7531FF75321B7533F5126CC47B047DDF
:103D430003E4FFF1BAF1D275320F75336A7B047D58
:103D530058E4FFF1BA752F0F75306C7531FF75326A
:103D63001B7533FE907FFFE493FFC4540FF534EFCC
:103D7300540FF5357B057D03E4FFF1BA752F0F75FD
:103D830030797531FF75321C7533077B067D03E48B
:103D9300FFF1BA752F0F75307E9080001209977866
:103DA30011120978EF541FFFE48F31120997781627
:103DB300120978EF540FFFE48F32120997781A1221
:103DC3000978EF543FFFEF24D0F534E43407F5339B
:103DD3007B067D3FE4FF124381301208E47872F6DC
:103DE300C212800930130678727601C213A210E45E
:103DF30033FF7872E67E00B401027E01EE5F600B52
:103E030012796CF1EA71E5D1D4C210124316816CB8
:103E1300227872E6FE08E690D80475F00A1209DCEF
:103E2300EE75F00AA42583F583E0FCA3E0FDA3E08F
:103E3300FEA3E0FF22301602C1D3123778D21690C8
:103E430087D712782A1279779087E9D12C126AECF6
:103E530090882FD12C90874DF1E3D12C908751126C
:103E630009D090882FD12C908743F1E3D12C9087F0
:103E7300471209D0127B149087D7D12C9087221236
:103E83006C98F89087D7D12C1208C7908729EF1226
:103E93004E489087D7D12C1208C7F1F1AF05908710
:103EA3002A124E479087D7D12C1208C7908728EB48
:103EB300F09087F2E0908726124E48908722D12C0B
:103EC3001208C7F1F1908727EDF01257F6123778F1
:103ED30022E4FBFD7C607F0351CBE4FB7D017C602E
:103EE3007F0351CBE4FB7D027C607F0351CBE4FB7A
:103EF3007D037C607F0341CB1278D4200802E1A3C9
:103F030090882FD12C90874DF1E3D12C90875112BB
:103F130009D09087E6E07002A3E0603B7E877F4D87
:103F23007C877D43126CE1E47FE87E03FDFC7871BE
:103F3300127A3A500280031278D490873BD12C1224
:103F43007895127971908737D12C127895908737AD
:103F53001209D0D20F802FC20FA20F300E01B3501F
:103F630025F1EA71E590873BE0FB7D00D1F5908771
:103F73003CE0FB7D01D1F590873DE0FB7D02D1F56F
:103F830090873EE0D1F290882FD12C908743F1E3C4
:103F9300D12C9087471209D0300F03D20E22C20EC4
:103FA30022852A82852983227531FF75321A75335A
:103FB300647B027D037F01124381752EFF22120071
:103FC3000EEF75F006A4FFC3743B9FFD752EFF75BE
:103FD3002F0E7530BF7531FF227480F074AAF02262
:103FE3001209D0908833227D007C607F03227C00FD
:103FF3007D6402079B90655574AAF0906AAA745574
:10400300F0906555228C658D66E4FEFDBF010A3193
:1040130046123FDC902AAA8024BF020A3136123F9F
:10402300DC904AAA8017BF030B123FF8123FDC90C3
:104033006AAA8009123A7D123FDC908AAA7455F06D
:104043008566828565837430F085668285658331F4
:104053002CBB80047E018005BA20027D01EE700333
:10406300EA60E6ED64017028AB04530380BB800271
:104073007E01BF01059025558013BF02059045556C
:10408300800BBF0305906555800390855574F0F050
:10409300AF062290849EE06073B4050890849C74FC
:1040A30001F08022781C7C847D017B017A84799ED7
:1040B3007E007F4012070B7E007F407D007B017AEC
:1040C30084795C120A2490849EE024FD603224FDEE
:1040D300602514601914601B14600924087028E417
:1040E300F5AE801790841B7401F0E4A3F022311025
:1040F300E48008311980043110311990841CF022B6
:1041030090849F31231108E4FF12399C2290849FED
:10411300E09000E0F0229084A0E09000E2F0E4223E
:10412300E0FFA3E0FCA3E0FD22E0FCFB5420FA53F4
:1041330003802290455574AAF0904AAA7455F090D2
:1041430045552290255574AAF0902AAA7455F090EB
:10415300255522C0E0C0F0C083C082C0D075D018FE
:10416300E5E830E111E5EA30E609E5ED54306003B6
:1041730053EABF53E8FDE5E830E45843EA3853EA2D
:10418300DF9084DEE0FFC394405043C374409FFF3D
:10419300C39408500280027F08789BEFF69084DE78
:1041A300E024DF127B4DEFFD7C0012747953E8EFBE
:1041B300789BE6FF9084DEE02FF0C3944040051225
:1041C3007685800F9084DEE0FF12399C800551884C
:1041D30053E8EFE5E830E37DE5ED30E61812760AC3
:1041E300789DEFF653E8F7E6606B1275CAEF7065DA
:1041F3001272958060E5ED540F605490849DE0C386
:104203009440504BE5ED540F789BF6087600789B6D
:10421300E6FF08E6FEC39F501490849DE02E249E83
:10422300F582E43484F583E5EFF00680E163ED8005
:1042330053E8F7123903789BE6FF90849DE02FF053
:10424300C394404010119653EA9043EA20800663DA
:10425300ED8053E8F7E5E830E2061274AD53E8FB6E
:10426300E5E830E00353E8FEE5E830E70353E87F91
:10427300E5E830E50553E8DF51B1D0D0D082D083F3
:10428300D0F0D0E03212738AEF7022908817E0B436
:104293000515A3E0FF4480F5EEEF90881F600574D9
:1042A30003F080037402F090881774FFF0221275F4
:1042B300BA75E10275EA3875EA1875EC0C75EB28E6
:1042C30075E6BA75E6BE75EB2275E9BF75EE80F546
:1042D300E875B70143A7012290881212667E908881
:1042E3000E1271D451EE12728880C37F01126041A5
:1042F3008021752F1A7530377531FF75321C753370
:104303001B908839E0F534A3E0F5357B057D05E4A2
:10431300FF7181E4FF12605DE47875F67875E6FF5E
:10432300C39408504D126069E47876F67876E6FF18
:10433300C394805038EFC394405009C2C5D2C4EF30
:104343007011800BD2C5C2C47876E6B44005E4FF91
:10435300126078D297C2C2D2C67876E6FF18E6F129
:104363006A2F1237C3E0126062080680BF787506B1
:1043730080AA2275321A75335C7B04E4FDFF8F2B10
:104383008D2C8B2DE4908767F0A3F0A3F0A3F07836
:104393007576280876F4F540754100754231852E0F
:1043A30043852F44853045854046854147854248AE
:1043B3007B017A8479021219BDF1C8FF7002A10D45
:1043C300E52B705DEF24E0908769F0A37406F0E4B9
:1043D300A3F0F17B400281FA908768E0FDE52C2D84
:1043E300FDE433FCEE7E002DFFEE3C127A834002A7
:1043F30081FA90876BE0F9908769E075F006A42451
:104403003DF582E5F0341CF583E582291237C3E4D8
:1044130093FD75F080E52DF16D1278DEEDF19C8052
:10442300B1E52B64017043F1C824E0127B1D24071E
:10443300F582E5F03424F1D7E490876BF0F17B50FB
:10444300211278A7501C12792DE58335F0F583C02E
:1044530083C08290876BE0FFD082D083F143F193D6
:1044630080DBF1C0640270D081FAE52B6402600244
:1044730081FAF1C8FF64206049EF24D0127B1D2428
:10448300F4F582E5F03428F1D7E490876BF0F17B03
:1044930050211278A7501C12792DE58335F0F5834E
:1044A300C083C08290876BE0FFD082D083F143F159
:1044B3009380DBF1C0640370D090876AE02402F03C
:1044C300803590876A740EF1F3E490876BF0F17B8B
:1044D3005020EE252CFFE433FE908768E07C002F0C
:1044E300FFEC3E127A83500AF1641278DEE4F19C09
:1044F30080DCF1C0B403D290876AE0FF908768E064
:104503002FF0908767E004F061BCE52B700890877B
:1045130068F1B9048012E52B908768B40106F1B9FC
:1045230024028004F1B92403FD0234318F277A2E4B
:104533007B5F752C037D037F67123354E527C454D7
:104543000F30010E7E00540FFF124F538E318F3206
:104553008003127A19752EFF752F1A7530257B0388
:104563007D6FE4FF7181E527540F14B40B00400203
:10457300C15B90457E126FC6C5837302459F02459A
:10458300B80245E30245FB0246130246360246489B
:1045930002465B024613024613024613D15C753191
:1045A300FF75321A753379E4FB7D1E7F0171817AC1
:1045B3002B7B67C158D15C7531FF75321A75338017
:1045C300E4FB7D1E123FB8D15F7531FF75321A755A
:1045D30033797B027D1E7F0171817A2B7BE98075A4
:1045E300D15C7531FF75321A75338AE4FB7D1E1277
:1045F3003FB8D1667B6B805DD15C7531FF75321A34
:1046030075339CE4FB7D1E123FB8D1667B6B8045FE
:10461300D15C7531FF75321A7533A3E4FB7D1E122D
:104623003FB8D15F7531FF75321A7533ADD1757BE4
:104633006B8022752EFF752F1A75302C1279F6D1E7
:10464300797B6B8010752EFF752F1A7530301279B8
:10465300F6D1797B6B12334F22752EFF752F1A75A6
:10466300302922752F1A7530297531FF75321A7565
:1046730033937B027D1E7F0171817A2C22908839CE
:10468300E0FAA3E0FBC39433EA94034002E11B90F6
:10469300882F123E2C90D800127AF9F1B2F58312CA
:1046A3003FE3123E2C90D804127AF9F1B2F583124B
:1046B30009D0908837E0C374809480500AF188AFA2
:1046C30005ED24B4FF8007908837F188AF05127198
:1046D3000290D80875F00A1209DCECF1B2F583EF09
:1046E300F090D809127AF0F1B2F583E4F090883AA9
:1046F300E004F07006908839E004F090883912677E
:10470300161270FB7531FF75321A7533CE7B0212A8
:104713003FB851F57F0A801812671D1270FB75317F
:10472300FF75321A7533D57B02123FB851F57F18E6
:104733007EB01256317F407E4B7D4C7C000250EFA1
:104743002582F582E43583F583740193FEEFFDE55D
:104753002C2DFDE433FC908768E07A002DFDEA3CC4
:10476300FC90876CE0252D75F080A42400F582E58C
:10477300F03480F583E5822290876AE0FFA3E0FEB0
:10478300C39F22F583E0FF7E007C007DB40207F027
:104793002DF582E5833CF583EEF090876BE004F022
:1047A30022E6FE08E6907FFE75F00A1209DCEE753C
:1047B300F00AA4258322E0252CFFE52D2290876CA7
:1047C300E004F0E022908767E02402F582E4348479
:1047D300F583E022F583740193FA740293AE02FF2A
:1047E3007875EEF608EFF6F5828E83E49390876A88
:1047F300F0E490876CF022C2AFD2A8C2B8C289D2CB
:10480300885389F0438902758CADE4F58AD2B9D215
:104813008CD2A9F5C8D2BD75CD6375CB6375CCC0F9
:1048230075CAC0D2ADD2CAC299C28E43878053899A
:104833000F438920758DECD28E90851FF0908520D3
:10484300F0759850C299C298D2ACD2BC75913075AC
:10485300950343972075948875B10875B20775B3AE
:104863000875B40775A131D2AF43A71022300C3CB1
:1048730090880DE025E025E04422F597E59730E0A8
:10488300FB90880DE0FF14600804700B908805808E
:1048930003908802E596F0EFC39401500890880DC9
:1048A300E004F08005E490880DF0C20C22C0E0C063
:1048B300F0C083C082C0D075D000C000C001C00268
:1048C300C003C004C005C006C007C2A878AA76000A
:1048D30020B20878AAE6D3942340F578AAE6D394C5
:1048E3002350213124EF601C3124EF60173124EF72
:1048F30060123124EF600D3124EF60083167908836
:104903003E7405F0D2A8D007D006D005D004D0035A
:10491300D002D001D000D0D0D082D083D0F0D0E06C
:1049230032E478AAF630B20878AAE6D3942340F5A5
:1049330078AAE6FFC3940E4028EFD394145022E4E0
:10494300F620B20878AAE6D3942340F578AAE6FFC6
:10495300C394004009EFD3940650037F01227F00E4
:10496300227F0022E4FF7E01FDE478AAF630B21232
:1049730078AAE6FCD394235009EC942340EF7EFFFE
:1049830080EBEF25E0FF78AAE6FCC3940B400BEC29
:10499300D3941150054307018013ECC39404400BD7
:1049A300ECD3940A50055307FE80027EFFE478AAF5
:1049B300F620B20878AAE6D3942340F578AAE6D382
:1049C300942340027EFF0DED6408709DEEF46010A9
:1049D30090883BEFF0E0C4540F7002C2207F0122A5
:1049E3007FFF22C0D075D008C28C78AA06D28CD0A3
:1049F300D032C0E0C083C082C0D075D01030981EC2
:104A0300C29890851FE02401FFE433FE908520E0E7
:104A13006F7001EE600890851F512AE599F0D0D0A0
:104A2300D082D083D0E032E0FF04F074212FF582EE
:104A3300E43485F58322908520E0FF90851FE0C351
:104A43009F70037FFF22C2AF908520512AE07872C6
:104A5300F6D2AFE6FF2251397871EFF6F4600FE634
:104A6300FF600B908621E0FE04F05193EFF0787124
:104A7300E6FFF46006EF6003B40ADB908621E06092
:104A83000C2421F582E43486F583E0FF227FFF22A4
:104A930074222EF582E43486F58322F1ED90876546
:104AA30004F0908621E024FBFF908765E0FEC39F1E
:104AB3005015A3E0FF5193E0FEEF6E908766F090F0
:104AC3008765E004F080DB908766E0FF12726090F8
:104AD3008621E0241FF582E43486F583E0B5071CC4
:104AE300908766E0FF127272908621E0241EF582A1
:104AF300E43486F583E0B507037F01227F00227843
:104B03007176FF752AFF752B00752C69752D00755D
:104B13002E067B017A8679221218D4EF701A519EE1
:104B2300EF60157145EF600C787176062016091257
:104B33003E388004E47871F6E4908621F07871E6DB
:104B4300FF22E4FFFEFDFC7872F1437876F14378AF
:104B53007A1209C47E867F22F19BB1A7F19BB1C66D
:104B63001203CB9087651209D0908765123E2C9073
:104B730087D71209D0F1A99087D7123E2C90875E70
:104B8300126C98F89087D7123E2C1208C79087634F
:104B9300EFF0E070037418F0D1499087D7123E2CE0
:104BA3001208C7123FF1AF05908764D1479087D7AA
:104BB300123E2C1208C7908762EBF078A6E6FE0837
:104BC300E6FFD12A908769B1B8D13FF16AF18DC070
:104BD30000787212098BD000F170787612098BE499
:104BE30012038D126CF1120169F1E51202721213B4
:104BF300FD7BCE7A6379DE7842120169D1591202C4
:104C030072D13F12016990872D1209D0F1801208E9
:104C13003CC004C005C006C007787212098BD003DC
:104C2300D002D001D000F1B8F178120169C004C0FC
:104C330005C006C007D150120169D003D002D001CC
:104C4300D00012007890876AD11990876EB1B8D1DD
:104C53003FF16AF18DC000787212098BD000F170B8
:104C6300F18012083CC004C005C006C00778721268
:104C7300098BD003D002D001D000F1B8F178120132
:104C830069C004C005C006C007D150120169D00332
:104C9300D002D001D00012007890876FD11990878D
:104CA30073B1B81203CBAD07AC06E41203927B18C1
:104CB3007A0979EDF168908774EEF0A3EFF04E6016
:104CC3000BE02405F0908774E03400F0F1A9B1A75C
:104CD30078A6A60608A607908774E07002A3E07082
:104CE3000A9087E8E0908776F0802778A4E6FE08AC
:104CF300E6FF78A7E624FFFD18E634FFFCB1E012D7
:104D03006CFA7C017D6812079BECC313ED1390874B
:104D130076F078A6B1BA1203CB9087771209D090B8
:104D2300876EE0B4530F90876A123E2C12037C9077
:104D3300876A1209D0908773E0B4570F90876F1278
:104D43003E2C12037C90876F1209D0C208908769AA
:104D5300E06441704C78D77C877D017B017A877949
:104D630065FE7F1612070B9087DC123E2C90882F6E
:104D73001209D09087E1123E2C9088331209D0900B
:104D830087E8E0908837F0E4A3F0D2089087D71241
:104D9300782A1279779087E9123E2C126AEC7F0108
:104DA300227F00220FEFAC0670010E14F5828C8374
:104DB300E0B42CF022F008E6FE08E6FF78A4A6068D
:104DC30008A607B1A778A6EEF6FC08EFF6FD78A4CF
:104DD300E6FE08E6FFED24FFFDEC34FFFC8E278F93
:104DE300288C298D2A787B7C877D017BFF7A30791B
:104DF300E27E007F0F12070BC3E52A9528FFE52902
:104E03009527FEAA27A9287B01787B7C87F1DD7A89
:104E130087797B0219371209D078A6E6FE08E6FFE8
:104E230078A4A60608A607B1A778A6A60608A6072B
:104E330078A4E6FE08E6F5828E83E022E4FBFA79A5
:104E43007A784422EDF0E47B64FAF9F8227876125A
:104E5300098BE412038DE4FBFA796178452290878C
:104E63009BE0FF12452F7E877F92125E4F7871126F
:104E7300098B126CE8752EFF752F1275305EF1F5F4
:104E83007B057D4B7F02123FBA752F127530638508
:104E93002A348529338528328527317B067D767F21
:104EA30001124381E47F64FEF12C500B752EFF75D4
:104EB3002F127530658067F13AD149D312096750D3
:104EC30013E47FC8FEF12C500B752EFF752F12755E
:104ED300306B804AF13AE47BC8FAF9F8D3120967D8
:104EE3005012E47F2CF12A500B752EFF752F12758B
:104EF3003071802AF13AE47B2C7A01F9F8D3120954
:104F0300675012E47F90F12A500B752EFF752F1214
:104F13007530778009752EFF752F1275307D7B05EF
:104F2300E4FD7F020243817E01FDFCAB2AAA29A98D
:104F330028A827C3020967AF2AAE29AD28AC2722C8
:104F43001209C4E4FFFEFDFC2290880CE0FF7E0002
:104F53007C007D0A120789AC06AD07E41203927B3D
:104F6300DB7AF9791E783F1201690203CB1208C775
:104F730078760209C4E4FBFA79707842227FA07E36
:104F8300867D017C0078760209A778721209C47BBA
:104F9300A07A86790178002278A6EEF608EFF678F3
:104FA300A4A60608F62278A6E6FE08E6FF78A4A6DD
:104FB3000608A60722C3EF9BFFEE9AFEED99FDECD0
:104FC30098FC787A1209C4787A12098BE412038D5B
:104FD300E4FBFA797A78440202727D0112070B7BB3
:104FE3000122E4FBFA7934784322E4908765F0A345
:104FF300F0228F348E338D328C3122C0E0C0F0C06A
:1050030083C082C0D075D008C2CF908804E4F0E595
:10501300C0F4540325E025E0FFE590F454034FF07A
:10502300E0FF908811E0FE6F6021EF600E90880F23
:10503300E4F090872004F0A374F4F090880FE0C3A9
:105043009496502FEE602C42228028EE60259087A4
:10505300207401F0A374F4F090880FE0FFC39496DA
:105063005002800CEFB4960BD214EE422290880FBC
:10507300E004F0908804E0908811F0908720E070BD
:1050830002A3E0600E908721E024FFF0908720E0E8
:1050930034FFF0908801E004F0E0C394324004E46C
:1050A300F0D20C908806123E2CEC4D4E4F601C90B3
:1050B3008806A3A3A3E024FFFFEE34FFFEED34FF35
:1050C300FDEC34FFFC9088061209D090883EE06026
:1050D3000214F0D0D0D082D083D0F0D0E0327F1B46
:1050E3007EB0D1317FC07EC67D2D7C008F2B8E2A72
:1050F3008D298C28E47F207E4EFDFCAB2BAA2AA9A8
:1051030029A828C31209674024E47B207A4EF9F8C2
:10511300AF2BAE2AAD29AC281208C7908806120916
:10512300D0908806123E2CEC4D4E4F70F42212792B
:10513300A3300111FCA3E0FD124F5E127B35124F29
:105143004CF1FC800A127AA290880CE0127A6D125C
:105153007B0B6052127A62404920184CD3ED944A7B
:10516300EC94015039123778752EFF752F13753073
:105173008D123FAB31B2127835400CF1D475307FCC
:1051830012788B7D5C80051278807D607F011243ED
:105193008112431611E111E111E1D218800AC218FC
:1051A3008006C2188002C2187F0122FD752EFF758A
:1051B3002F127530237531FF228F271267FBC3909F
:1051C30087E7E0944A9087E6E09401400F90872BAD
:1051D300E0FFA3E09087E6CFF0A3EFF0E5276402BA
:1051E300600241FB31AF75321A75335CFBFDFF1270
:1051F300438130011B127AC0F1EEFD124F5E8E31F6
:105203008F321279B2752EFF752F1275309F801170
:10521300127AC0F1DB1279B2752EFF752F12753039
:10522300A31267E531AF75321B7533B312437C901C
:1052330087E8E0F4700241E6E0FF740BD39F50115E
:10524300E0C39421500B752EFF752F127530A741C3
:10525300F21269615011E0C39438500B752EFF753B
:105263002F127530AE41F21269575011E0C3944EBC
:10527300500B752EFF752F127530B5807212694D64
:105283005011E0C39465500B752EFF752F127530C6
:10529300BC805C1269435011E0C3947B500B752EA4
:1052A300FF752F127530C380461269395011E0C360
:1052B3009492500B752EFF752F127530CA803012E1
:1052C300692F5011E0C394A8500B752EFF752F1250
:1052D3007530D1801A752EFF752F127530D89087CF
:1052E300E8800C752EFF752F127530DF9087E8125A
:1052F300696B7D0A7F02C109E52764016002A13160
:1053030031AF75321B75338D7B01FDFF1243813045
:105313000116752EFF752F127530E6F1AE908737A3
:10532300123E2C1277FE8012752EFF752F127530E8
:10533300EF908737123E2C124FCF124FF57B017D32
:105343002CE4FF12438131AF75321C7533377B0276
:10535300E4FDFF123FBA752F127530F8908726F1DE
:10536300DE7B027D1CE4FF123FBA752F13753003F9
:105373007531FF7532137533109087F2E0F534A35E
:10538300E0F5357B027D3AE4FF123FBA31B2753264
:105393001B7533BC7B03F1A8300116752EFF752FE7
:1053A30013753012F1AE90873B123E2C1277FE80BC
:1053B30012752EFF752F1375301B90873B123E2CF1
:1053C300124FCF124FF57B037D26E4FF1243813149
:1053D300AF124376300115752EFF752F13753024E8
:1053E300F1EEFD124F5E8E318F32800B752EFF75FD
:1053F3002F1375302CF1DB7B04127B559087291218
:105403006A001278FE908728E0FFE4FEEB2F127803
:105413009C90873F1209D0908763126A001278FE2E
:10542300908762E0FFE4FEEB2F12789C90871C12BA
:1054330009D090873FF1C890871C12782AC39BFF3D
:10544300EE9AFEED99FDEC98FC9087571209D03146
:10545300AF75321C7533317B05F1A8908737123E47
:105463002CEC4D4E4F604330011A127AB6127A7803
:10547300F1C812083C908757F1C81208C7F1AE1261
:1054830077FE801C127AAC127A78F1C812083C902D
:105493008757F1C81208C7F1AE1208C7E412038D8B
:1054A300124FF57B057D2CE48012300105127AB68C
:1054B3008003127AACE4F5317B057D2CFF12438126
:1054C30031AF1267DE7B06F1A8127A2330010D1289
:1054D3004F57F1E6752F13753024800B120789F1AE
:1054E300E6752F1375302C7B06127B5531AF753261
:1054F3001B7533C07B07F1A812672E752F13753008
:10550300489087F0E0F5319087EFE0F5327B07E4D0
:10551300FF123FBA752F137530527531FF75321371
:1055230075335D126CC47B077D4BE4FFC10931AF5A
:1055330075321B75338DE4FBFDFF12438130011679
:10554300752EFF752F13753061F1AE908737123EBC
:105553002C1277FE8012752EFF752F13753069900C
:105563008737123E2C124FCF124FF57B017D2CE46F
:10557300FF12438131AF1267DE7B02F1A890880CE2
:10558300E0FF602630010D124F51F1E6752F1375C0
:105593003071801090880CE0127A19752EFF752FE8
:1055A300137530787B037D3280137BFF7A1A79720F
:1055B3001279EDFFC3745A9F31AE127ADEE4FF1203
:1055C300438131AF124376300120F1D475307FF13E
:1055D300EEFD124F5E8E318F327B057D2D7F0212E1
:1055E3003FBA752F1275309F8016F1D475307FF155
:1055F300DB7B057D2D7F02123FBA752F127530A319
:105603007B067D5E7F011243819087F2E0FF9087E6
:1056130032E06F6002F1F6127B149087E6E0FFA39D
:10562300E090872BCFF0A3EFF0227F1D7EB03002F6
:1056330014D374189F74B09E500BEF941EEE94B065
:1056430050037F00227876A60608A60720B7FDD26E
:10565300B5C2B4C2B60000E47875F6127B2DEE3005
:10566300E704D2B48002C2B4C2B5EF25E07977F77C
:10567300EE3319F70000D2B50000787506E6B410D2
:10568300DAC2B40000D2B630B7FD7F0122752EFF17
:10569300752F137530937B017D13E4FF123FBA75A9
:1056A3002F1375309C7B027D117F02123FBA752F39
:1056B300137530A47531FF75321B7533C57B057DBA
:1056C3001C1243122002111279137F0C7EB0D131C8
:1056D3007FC07EC67D2D80067F807E847D1E7C00FC
:1056E30011EF90883EE060127F1FF1037F20F103EA
:1056F3007F21F1037F227EB0D131126D13023778FF
:105703007EB0D1317F807E847D1E7C0001EF8F27A8
:105713001279A330011BFCA3E0FD124F5E127B350F
:10572300E527C4540F7E00540FFF124F53F1FC8042
:105733000B127AA2E527C4540F127A6D127B0B6009
:105743005F127A624056201959D3ED942CEC9401E0
:105753005046123778752EFF752F12753023123F7E
:10576300AB752F137530837531FF127835400CF10B
:10577300D475307F12788B7D5C80051278807D60D4
:105783007F011243811243167F1A11E37F1A11E33B
:105793007F1A11E3D219800AC2188006C219800247
:1057A300C2197F0122E4FDFF024381E47BE87A030F
:1057B300F9F8221209DCEE75F00AA42583F58312A9
:1057C300099790882FE0F8A3E0F9A3E0FAA3E0FBA0
:1057D30022752EFF752F13229087E6E0F531A3E0A3
:1057E300F532228E318F32752EFF229087E6E0FC50
:1057F300A3E0227F1E7EB0C1317871A60608A607FA
:10580300227F01124381752A017B7FE4FDFF7874B7
:10581300A6077874E6D39B503EE52A7018F1CD12A3
:10582300476D2F1237C3E044021279411237C3E0A8
:105833004440F0801DE52A640170177874F1CD129D
:10584300476D2F1237C3E0F41279411237C3E06476
:105853007FF078740680BB22E47872F608F6301184
:1058630002413290841BE060024132908400E0FDEB
:10587300752EFF752F0E7530EA7531FF75321A7567
:1058830033C7E4FB7F01124381908839E07002A3A0
:10589300E0701A752A017B7FFDFF1111123FCF754E
:1058A300321B7533DB7B047D19E4FF21EA752EFF80
:1058B300752F0E7530FA7873E62401F53218E43645
:1058C300F531E4FB7D66110478725135123E1D51AA
:1058D3003D7872600250075135123E1D80085135E4
:1058E300123E1D12037C124E591279DFF078725169
:1058F30035123E1D513D9087D5600250105147C06F
:1059030004126A1078725135123E1D801A5147C035
:1059130004C005C006C00778725135123E1D12033C
:105923007CD003D002D001D00012791A787251359D
:10593300123E1D513D7F53600250027F4E8F3175E1
:105943002EFF752F0F75300012781DF537126CDAA4
:105953007B02F1D4123E14513D787260025005125D
:105963003E168006123E1612037C124E591279DF40
:10597300F0123E14513D9087D56002500C5147C040
:1059830004126A10123E1480165147C004C005C0A9
:1059930006C007123E1412037CD003D002D001D0FC
:1059A3000012791A123E14513D7F57600250027F54
:1059B300458F31752EFF752F0F75301912781DF530
:1059C30037126CDA7B04F1D47872F1DB1247ABF552
:1059D30083E075F002127A1C752EFF752F0F753058
:1059E300327B067D077F01124381126387301317D1
:1059F300D37873E6940018E69400400708E6161877
:105A0300700116C2130161201202016190883AE00D
:105A130024FFFF908839E034FFFEC37873E69F18B4
:105A2300E69E50070806E618700106C212016122BD
:105A33007875E6FE08E690D80022E4FBFAF9F874DC
:105A4300F0020311E0FEA3E0FFE4FCFD7B107A0EFD
:105A5300F9F812083CE402038D908839E07002A340
:105A6300E070026163E47875F608F67875D1361252
:105A7300710B9E5002616390D80075F00AEF123EDD
:105A830020127A2F1257C574F01203115002615974
:105A93005133123E1DF1FB1257C574F0120311600E
:105AA30004400261597875123E167B927AB17909E6
:105AB30078C2D1EC1257C874F01203115002615925
:105AC3007875123E167B927AB179097842D1EC123D
:105AD30057C874F01203116002507B51331247AB65
:105AE300AF82FE7C887D2F126A177877A607E6FFC0
:105AF300F46063908837E0FB71F7605A7875E6FECF
:105B030008E6FF90D8081247ABF583E0C37480948E
:105B130080501590D80875F00AEF1247AE124786E9
:105B2300AF05ED24B4FB800E7875F1DB1247AB12A1
:105B33004786AF05AB07787771F5601A5133124783
:105B4300ABFAA9827B0178237C88D146E490882C28
:105B5300F07876026EEF787606E618700106416EED
:105B6300126F29E4FEFF228F2CAA05127A41C36427
:105B7300809480500912478CED24B4FF8008127A78
:105B83004112478CAF05788FA607EA252CFFE43333
:105B9300FEC364809480500912478CED24B4FF80C7
:105BA3000CE52C2AFFE433FE12478CAF057890EF07
:105BB300F618E6FEB507037F01227890E6FFEED3E1
:105BC3009F401B18E6D39B5006EBC394B44009E4F3
:105BD300D39B5007EB9F50037F01227F0022788FD6
:105BE300E6D39B500A08E6FFEB9F50037F01227F19
:105BF3000022E6FF7D16716AEF22F1F3F1BDF1E3B6
:105C0300E408F608F608F608F6F1B6081209C4F136
:105C1300B67882124F4378861209C4126E3F787A9F
:105C2300EEF608EFF6D39414EE94005004F1F380EB
:105C33000A787BE624EC7977126EE7F1BDFF24EC5A
:105C4300FDEE34FFFC787AE6FA08E6FBC39DEA9C96
:105C530040097878A60608A607800AEB2414787909
:105C6300F6E43A18F6F1BDFF4E7002C130EB4A700C
:105C730002C1307878EAF6FC08EBF67876A60408D9
:105C8300F64A6006E61618700116EF6B7002EE6AAC
:105C93006008787906E618700106D37877E69401F0
:105CA30018E694004026787A1247A4F583120997E0
:105CB300127A2F78761279941247B2127A4D600CC9
:105CC300400A7877E6161870011680CE7878D136B8
:105CD3009087B7E09F9087B6E09E4022081247A4C2
:105CE300F583120997F1FB78781279941247B2126F
:105CF3007A4D500A787906E61870010680CE127B39
:105D03002D787AA60608A607787AD136787996EEA2
:105D130018965078907FFE75F00AEF1247AED13D8A
:105D23009087A4E0B4EE03127B027E877F9C7C887D
:105D33007D2F126977787E1209C47E877F9C126D4E
:105D430006F4603E908837E0FB71F760359087A4D6
:105D5300127A98500912478CED24B4FB800A90877D
:105D6300A4124788AF05AB07787571F56014F1EBA2
:105D7300123614400DF1EB1209C4787AE6FE08E6F8
:105D8300F1E3787B06E618700106A10B787DE6182F
:105D9300467002C130E47F207E03FDFC7882127AD4
:105DA3003A4002C130787C1247A4D13D9087A4E0E9
:105DB300B4EE03127B027A877B9C7D0F7FBC7E024D
:105DC3001236F078861209C4F1B67886123614605A
:105DD3005CE4FFFEFDFC788612361460509087B9B0
:105DE300E0FFE4FCFDFE7BCC7A0CF9F812083CEFF3
:105DF300787D26FFEE1836FE787AF608EFF6908760
:105E0300A6E06E7003A3E06F6023787AE6FF08E6EE
:105E13009087A6CFF0A3EFF07A87799C7B017892E5
:105E23007C87D1469087A6E0FEA3E0FF22E4FEFF35
:105E3300227876E6FE08E6FFD322FAA9827BFF7872
:105E43009C7C877D017E007F0A02070B126D069002
:105E53008837E0D39F4012EF24B4FFE433FEE0FD24
:105E6300C3EF9D7877F6EE800E908837E0FF787564
:105E7300E6C39F7877F6E4940018F6D134740B9F49
:105E8300E49E500FC3EF9421EE940050067A2E7BCC
:105E930015804CD13474219FE49E500FC3EF943886
:105EA300EE940050067A2D7BCB8034D134747B9FE3
:105EB300E49E500FC3EF9492EE940050067A2D7B2C
:105EC30081801CD13474929FE49E500FC3EF94A839
:105ED300EE940050067A2D7B3780047A2C7BED7587
:105EE3002C03E4FD7F670233541200789088332239
:105EF300908839E07002A3E07002E1AF124FED1217
:105F03007AE7908765E0FCA3E0FDC39FEC9E400227
:105F1300E1AF90D800127AF0123E247B1C7A3479D8
:105F23004F78C01200781257C574F0120311406CF9
:105F3300F1C590D800123E1D7B1C7A34794F78400E
:105F43001200781257C574F01203116002504DF11C
:105F5300C590D804123E1D7B927AB1798978C0D15D
:105F6300EC1257C874F01203114031F1C590D804F4
:105F7300123E1D7B927AB179897840D1EC1257C8D1
:105F830074F012031160025013908766E02401FF3E
:105F9300908765E03400FE12704B8013908766E0B3
:105FA30004F07006908765E004F0E102124680E495
:105FB300FEFF2274FFFFFEFDFC229087B6E0FEA3E6
:105FC300E022908765E0FEA3E022E6FF75F080ED16
:105FD300227D077F01024381E6FE08E690D808226E
:105FE300FF08A60608A60722787E12098B7882226C
:105FF30078767600087601227B1C7A3479CF784153
:106003000200787873A6077873E6FFD39B502EE5DA
:106013002A701175F080ED12476D2F1237C3E044DB
:1060230002F08014E52AB4010F7873125FCD124792
:106033006D2F1237C3E0F4F078730680CA22D2972B
:1060430000115400EF443E900005F000C29722D2A5
:1060530097C2C2C2C6D2C5D2C4221152EF44C09065
:106063000005F0C29722AE071152EE44B8116290B8
:106073008401EEF022AE07D297C2C2C2C6EE4440FC
:106083001162908400EEF022E47871F67871E6FFF5
:10609300C394FA500B74222F124A96E4F00680EC54
:1060A30022300814A210B014500E9087E8E0F46078
:1060B30005511A125EF3C210A211B0145007123721
:1060C300F711DD800FA2137212500CC212C2131209
:1060D3003778B1DA12377802002630110241029084
:1060E300841BE060024102908720E07002A3E0700D
:1060F300024102E49087D4F0123FCF75321A753310
:10610300E9FBFD7F01124381E47871F67871E6FFC4
:10611300D3947F500C7B407D0112346778710680E5
:10612300EBE47871F651125039EF7168FDEF715954
:10613300FCEF510375F012A424C4F9740FD1861235
:1061430043817871E651037149B50611E6FE716822
:10615300FFEE7159FD752A017B7F12581178710684
:1061630080C312431630133D511A9087D1E0D39464
:1061730000402EE014F0E47871F65112500FEF5105
:10618300037149B50602714278710680ED713B6077
:1061930010E47871F651125008EF510314F00680A1
:1061A300F4C213803E30123B511A9087D1E0C3945E
:1061B30005502EE004F0E47871F65112500FEF51C0
:1061C300037149B50602714278710680ED713B6037
:1061D30010E47871F651125008EF510304F0068071
:1061E300F4C21220100201DD1237F79087D1E07557
:1061F300F003A42463F582E4341012376701DD222F
:1062030075F003A424C7F582E43487F583E022788C
:1062130071E6FFC39403227F197EB0025631301119
:1062230002612390841BE0600261239087D4F0D144
:106233009475321B753324E4FB125804E47872F628
:1062430071335040EF75F003A424BFF582E4348723
:10625300F583E0FD7177FCEF712475F011A4243010
:10626300F97410D1861243817872E6FF7124FE908F
:1062730087D0E0FDEEB505077177FB9167718C78E8
:10628300720680BC718730133D511A9087D0E0D3DA
:106293009400402EE014F0E47872F67133500FEF5F
:1062A30071247151B50602714278720680ED713B1B
:1062B3006010E47872F671335008EF712414F0061D
:1062C30080F4C213803E30123B511A9087D0E0C352
:1062D3009402502EE004F0E47872F67133500FEF1D
:1062E30071247151B50602714278720680ED713BDB
:1062F3006010E47872F671335008EF712404F006ED
:1063030080F4C21220100241211237F79087D0E0A7
:1063130075F003A42475F582E43410123767412124
:106323002275F003A424BEF582E43487F583E022CA
:106333007872E6FFC39403229087D4E0640122902D
:1063430087D47401F022FF9087D1E0FEEF22FF9003
:1063530087D0E0FEEF2275F003A424C9F582E4346C
:1063630087F583E02275F003A424C8F582E434871B
:10637300F583E022EF75F003A424C0F582E43487AB
:10638300F583E02291D70243167D057F0102438105
:10639300E47872F690880BE0F6301102815F908406
:1063A3001BE06002815F908400E0123FCE75321AD9
:1063B3007533F8E4FB12580430131290880BE0D3C2
:1063C30094004005E014F0D209C213801330121078
:1063D30090880BE0C394025005E004F0D209C21286
:1063E300752EFF91CD75321B7533947B027D05129B
:1063F3003FB891CD75321B75339B7B047D05123FEE
:10640300B891CD75321B7533A37B06718C90880BC5
:10641300E0700691677B02801890880BE0B4010658
:1064230091677B04800B90880BE0B4020691677B35
:1064330006718C301022C21090880BE07872F6122D
:106443003778F11D123FD275321C753310F1E51206
:1064530043161250E71237787187619C7872E69081
:10646300880BF022752EFF752F0E7530C62290848F
:1064730000E0123FCE75321B753353E4FB12580410
:1064830091D720114490841BE0703E301206B1C9AD
:10649300C2128007301304B1C9C213752EFF752FC2
:1064A3000F75308A7B037D05123FB8752F0F75304A
:1064B300987B05718C20010691677B0380049167AB
:1064C3007B05718C12431680B922752F0E7530C26D
:1064D3007531FF22E47874F67874E6FFD3947F5025
:1064E3000C7B807D0712346778740680EB787476B2
:1064F300017874E6FDD3940750177BFFE4FF123451
:10650300677874E6FD7BFF7F7F12346778740680BB
:10651300E022D194F1DEE4FB12580491D73011024A
:10652300A1C890841BE06002A1C830121290880CAD
:10653300E0C394215005E004F0D209C21280133065
:10654300131090880CE0D394004005E014F0D209B6
:10655300C213752EFF752F0E7530CC7B03718C9093
:10656300880CE0604E200113752EFF752F0E7530D9
:10657300DCB1D1127A23120789800E752EFF752F95
:106583000E7530E4B1D1124F4C1257E6752F0E75CC
:1065930030E07B037D1E7F01124381752EFF752F33
:1065A3000E7530E87B037D0A123FB8916A7B037D49
:1065B3006E8008123FCF127ADE7D087F011243817D
:1065C300124316A12022A201B39201D209227B0316
:1065D3007D467F01024381908400E01251AE753203
:1065E3001A75333DE4FB12580491D7301002C17A77
:1065F30090841BE06002C17A908720E07002A3E0E0
:106603006075301214908812E0C3940A5004E004B9
:10661300D17B12562DC2128015301312908812E0CE
:10662300D394004004E014D17B12562DC213752E6F
:10663300FF752F127530269088121271BA123FB867
:10664300752F1275302B1271C6123431E47871F63E
:106653007871E6FFC3940A50199088121271AF50F3
:10666300067A297BA580047A297B8FF1F37871065A
:1066730080DE124316A1EE22F0D209E09030CC93D3
:10668300F5A22235F0752EFFF52F8930AB047F017B
:1066930022908400E0FD752EFF752F0E7530C875AE
:1066A30031FF22D19475321B753378E4FB12580401
:1066B30091D720114590841BE0703F301206D1FE24
:1066C300C2128007301304D1FEC213300210F10648
:1066D3007533747534FF75351A753672800EF1068D
:1066E3007533747534FF75351A75366B7B037D0A04
:1066F3007F0112438112431680B822A202B3920291
:10670300D20922752EFF752F0F7530BE7531FF75B7
:10671300321B22E0FEA3E0FFF1391234757A297BA4
:10672300BB752C037D027F0A123354908400E0244E
:1067330005FD752EFF228E278F287C407D007F026A
:10674300123BE57C407D00908839F1987C407D01C7
:1067530090883AF198E47873F608F6AE27AF287C70
:10676300007D0A120789C37874E69F18E69E5024B9
:106773007E40E6FA08E6FB2402FD74403AFC74000E
:106783002BF58274D83AF583F198787406E618707D
:10679300010680C722E0FB7F02023ACB78397C886E
:1067A3007D017B017A407900F1EC127AE74E602A91
:1067B300C3EF9433EE940350167C007D0A120789CD
:1067C30078007CD87D017B017A40790202070BE4D3
:1067D300908839F0A3F0FFFEF1392275321B75332F
:1067E3000A227B027F010243817E007F0202070BA4
:1067F300752C037D050233547A297BDD752C03E464
:10680300FD7F621233549087E8E0F470022115E0B3
:10681300FF740BD39F501DE0C3942150177A2B7B39
:10682300013127311D70022115752EFF752F127549
:10683300302D210931615022E0C39438501C7A2A4B
:106843007B79752C037D017F6B311D7002211575DA
:106853002EFF752F1275303321093157501DE0C3B8
:10686300944E50177A2A7BDF3127311D7002211590
:10687300752EFF752F127530392109314D501BE0EC
:10688300C3946550157A2A7B9B31167002211575C6
:106893002EFF752F1275303F806C3143501BE0C3C0
:1068A300947B50157A2B7B453127311D6064752EFF
:1068B300FF752F12753046804D3139501BE0C3945C
:1068C3009250157A2A7BBD3127311D6045752EFF05
:1068D300752F1275304C802E312F5019E0C394A8B8
:1068E30050137A2B7B2331166028752EFF752F12D8
:1068F30075305280117A2A7B5731166015752EFF39
:10690300752F127530589087E8316B7D61E4FF1263
:10691300438122752C037D017F6A12335490880BC7
:10692300E0640222752C037D017F69229087E8E0F1
:10693300FF7492D39F229087E8E0FF747BD39F225A
:106943009087E8E0FF7465D39F229087E8E0FF74A7
:106953004ED39F229087E8E0FF7438D39F2290871D
:10696300E8E0FF7421D39F22E025E0F532E433F51C
:10697300317B052291A2E4FFFEFDFC788F124F4389
:106983007893124F4378971209C4852F82852E83FB
:106993001257C8852D82852C83123E2C1200747BDE
:1069A3009A7A1979F77841120169789391B5125758
:1069B300C891AB123E2A12007490872D1257C81249
:1069C300016978971209C4789712098B510E120145
:1069D30069C004C005C006C007789312098B510E25
:1069E300120169D003D002D001D00012007812172F
:1069F3003591FA788F1209C4788F02098BE0FF7EF4
:106A0300007C0E7D10120789E4FCFDA804A905AAE9
:106A130006AB072291A2852F82852E831257C88F3A
:106A2300828E83123E2C120074788F91B51257C850
:106A330091AB123E2A12007478931209C478931210
:106A4300098B91D8788F12098B121861124FE512B6
:106A5300016991F1120272510EE4FFFE7DE17C4364
:106A63001200741203CB7897EEF608EFF651C95073
:106A73000D1851E0ED2468FFEC3401FE800B78978C
:106A830051E0ECC313FEED13FF7897A60608A607A3
:106A9300E4FFFEFDFC789351D0700DFFFEFDFC7802
:106AA3008F51D070037FFF2251D851C97D0050020E
:106AB3007D01ED600912478CED24B4FF800751D8A6
:106AC30012478CAF0522C3EE64809480221209A77B
:106AD30074F00203117897E6FE08E6FF22E6FE084B
:106AE300E6FF7C017D680207F091E8124E49120827
:106AF300C7EB24D0FEEA34079087EDF0A3CE124E05
:106B030048124F3A1208C7123FF19087EFEDF09108
:106B13009BF8124F3A1208C79087F0EFF0919BF859
:106B2300917E9087F2EF124E48917E123FF190874B
:106B3300F3124E47917E9087F4EBF0916654037005
:106B430018FC7D6412079BED4C700891669189EDEA
:106B53004C70069087F6741DF09087F2E0F9FF33CE
:106B630095E0FEAD2FED3395E0FCEF2DFFEE3CFEFF
:106B7300C3EF9418EE648094804026916FFD908754
:106B8300F0E004F0D39D40119087EFE004F0A3E020
:106B9300FD916FFCED8CF091909087F2E0252F80B2
:106BA3002751C950299087F0E014F09400501190B8
:106BB30087EFE014F0A3E0FF916FFEEF8EF091906A
:106BC3009087F2E0252F241875F01884800AE52FAA
:106BD3002975F018849087F2E5F0F09087EDE0FADC
:106BE300A3E0FB7C017D6DFFAE02120789AC06AD0D
:106BF30007EBAE027802CEC313CE13D8F92DFBEC0C
:106C03003E9165123FF1C3EB9FFBEA9E916591892B
:106C1300EF2BFFEE3ACF2494CF34FEFE7C007D07AA
:106C230012079B9087F1EDF0787E76019087EFE075
:106C3300FF787EE6FEC39F501574F42E9175FF9086
:106C430087F1E02F75F00784E5F0F00680DE90878A
:106C5300F1E014FF9087F0E02F75F00784A3E5F0CF
:106C6300F022FA9087EDE0FEA3E0FF229087EFE0A9
:106C730024F4F582E43487F583E022AF2EAE2DAD04
:106C83002CAC2B0208C77C017D9002079B84908764
:106C9300F0E5F0F0221209D0E47B107A27F9228E76
:106CA3002C8F2D8C2E8D2F22E52D2404F582E43597
:106CB3002C221209C4E52F2404F582E4352EF58332
:106CC30022908802E0FCE41203977B857AEB79C774
:106CD300783D1201698F378E368D358C34223177AA
:106CE30078710209C48F2A8E298D288C27227BDC98
:106CF3007A0F7949784022E4FBFAF9783F12007859
:106D03000203CB7C887D2F51177875A607E6FF22F7
:106D1300E4F527902975B18E7A297B75B17EB1860A
:106D230040F1124316B19AE4F527902982B18E7A85
:106D3300297B82B17EE47FD07E07FDFC1250EF12E7
:106D43004316B18640E4752EFF752F137530AB756E
:106D530031FF75321B7533D17534FF75351B7536AD
:106D6300AB7B057D1712431220020C7F007EB0120D
:106D7300563130B70580FB12570722752C037D0669
:106D83000233540527E527C3940922E493FFE5273B
:106D93008FF0A4240FFF22E47F107E27FDFC025016
:106DA300EF8F27E47872F6D1174527F0D2AF7A80B8
:106DB30079067BFFC001E52775F002A424A6F974C8
:106DC3008735F0A801FC7D01D0011267ECD109E001
:106DD300FEA3E0FFF47002EEF46004EF4E700BD1FB
:106DE30009E4F0A3F07872F6800478727601D10991
:106DF300E0FEA3E0FF9087B7E02FF09087B6E03E78
:106E0300F07872E6FF22E52725E024A6F582E43434
:106E130087F58322C2AF9000E0E054F822787176C0
:106E2300017871E6FFD394075011B1A4EF6007789E
:106E330071E69087B8F078710680E622E4788AF6E6
:106E430008F6125FBDFF24FF788DF6EE34FF18F6C7
:106E5300EF4E7002C1E3788CE6FE08E6FF788AE61F
:106E6300FC08E6FDD39FEC9E5072ED2FFFEC3EC372
:106E730013FEEF13FF788EEEF608EFF608A606086A
:106E8300F66D7002EC6E6054788EE6FE08E6FF78CD
:106E93008D66700318E66E604390800875F00AEF04
:106EA3001257B674F0120311500B788FE624FF7952
:106EB3008DD1E780A1788EE6FE08E690800875F014
:106EC3000A1257B674F01203116011400F788FE65F
:106ED3002401798BF718E43619F7C1597891800C9E
:106EE300E4FEFF22F718E634FF19F722E62401FF38
:106EF30018E436FE22E49087A6F0A3F0C21DC21E5A
:106F0300C21FC219FFFEFDFC908792F12090879665
:106F13001209D090879A74FFF0E4A3F0221209D0EB
:106F2300E4FFFEFDFC22F14AC21BC21CC21AFFFE93
:106F3300FDFC908823F1209088271209D090882B9C
:106F430074FFF0E4A3F022E490882DF0A3F022F183
:106F5300CF94004061ED605E14B40B005058906F05
:106F630069F1C6C58373026F8A026F8E026F920244
:106F73006FA2026F96026F9A026F9E026FB9026F41
:106F8300A8026FAE026FB27F0180167F0280127F6C
:106F930004800E7F03800A7F0680067F0780027FBE
:106FA300057EB0800E7F307EB48008F1BA8004F194
:106FB300BAF1BE125631227F307EB41256317F3081
:106FC3007EB42275F003A4C58325F022EF540FFD90
:106FD300EFC4540F75F00AA4FEFFC39087E7E09F48
:106FE3009087E6E022F1CF9400405CED14B40B00EF
:106FF3005055906FFDF1C6C5837302701E02702059
:1070030002702402703002702802702C02702C026D
:10701300704A02703602703C02704180007F0F801C
:107023000E7F10800A7F1080067F0D80027F107E06
:10703300B080117F307EB4800B126FBA8006126F5E
:10704300BA126FBE125631223102D39400EC94006F
:10705300500201DA90882DE0B50608A3E0B50703D6
:10706300126F4AED6F7002EC6E6041EF64014E6087
:107073003B1257FC7871125E36310B9E402E7C001A
:107083007D0A12078974002FF974D83EFA7B01C078
:107093000174F62FF974D73EA801FC7D01D00112CB
:1070A3005E48787206E61870010680C890883AE058
:1070B30024FFF0908839E034FFF012671611FB7556
:1070C30031FF75321A7533DB7B02123FB81242F57A
:1070D3007F0B124733801E12671D11FB7531FF753D
:1070E300321A7533E47B02123FB81242F57F18124D
:1070F30047337F00227F0122752F1A753034229087
:107103008839E0FCA3E0FD2290883AE09F9088391B
:10711300E02230110221AE90841BE0600221AE1206
:10712300669475321B753311E4FB12580430121444
:1071330090880EE0C3940A5007E004F0D20931D4DA
:10714300C212802030131D90880EE0D394004012A9
:10715300E014F0D209E09030D793FFF5AA74FF9FB3
:10716300F5ABC213752EFF752F0F75303E90880E49
:1071730031BA123FB8752F0F75304331C61234310F
:10718300E47872F67872E6FFC3940A501990880E79
:1071930031AF50067A297BA580047A297B8F126749
:1071A300F378720680DE124316211522E0FEEFC348
:1071B3009E908400E0FF22E075F00AA4F5317B0382
:1071C3007D4B227B037D647F011243817D057F0A12
:1071D30022E09030D793FFF5AAC374FF9FF5AB224B
:1071E30012669475321B753365E4FB1258041264FE
:1071F300D720116890841BE07062301214908803CA
:10720300E0C36480948C5005E004F0D209C212807C
:1072130015301312908803E0D3648094744005E022
:1072230014F0D209C213908803E0FFC364809480F2
:10723300400D752EFF752F0F7530A88F31800F7598
:107243002EFF752F0F7530B3908803E0F5317B0364
:107253007D197F0112438112431680952253070F34
:10726300EFD39409EF50042430FF222437FF225335
:1072730007F0EFC4540FFFD39409EF50042430FFF9
:10728300222437FF22D2B5D2B6C2B4D2C32275EAC2
:10729300B022B1BAA3E05460701AA3E024FB600EDD
:1072A30014600D24FD600B2408700902002E80DE9B
:1072B3008006815943EA4022908819E024FE602227
:1072C30014602D24E2605614606324217078913693
:1072D3007430F0A3741EF0908814E4F0A37412F0D9
:1072E300806891367430F0A3743AF090303C803962
:1072F300908818E075F003A424C3F582E5F03430D8
:10730300F583E493FB740193FA740293F990882054
:10731300EBF0A3EAF0A3E9F0120731801E91367473
:1073230030F0A37431F0903030E493800E913674D2
:1073330030F0A3745FF090305EE493FF908814E420
:10734300F0A3EFF0800443EA402290881DE0FE9012
:10735300881CE0FDEDFF789EEEF6FE08EFF69088C0
:1073630014E0FCA3E0FDC3914F7F0050027F019026
:107373008813EFF0789E125E36ED914F4006A3EE30
:10738300F0A3EFF053EA7F908820A3E0FAA3E0F99B
:10739300EA4970028130908814E0FEA3E0FF4E704A
:1073A300069146F5EA807A78A2EEF608EFF6D391D5
:1073B3003E40061876000876089146FF78A3E64F0C
:1073C300F5EAE478A0F608F6C379A1E778A396185E
:1073D300E66480F819E7648098501F908820E0FBEA
:1073E300A3E475F001120826A9F0FA120731F5E7B4
:1073F30078A106E61870010680CE78A2E6FE08E6BC
:10740300FFC3908815E09FFD908814E09EFCF0A3D5
:10741300EDF04C7015908813E06006C3EF913E5079
:1074230009908820E4F0A3F0A3F07F012275EA908D
:107433007F002290882074FFF0A3229408EE6480DA
:10744300948022E5EA648054804430229FEE648075
:10745300F8EC64809822908818E0D3940090881FF9
:1074630040077404F0917380037403F075EAB0224B
:1074730091AD53EADF228B658A668967D3ED940861
:10748300EC6480948040047C007D0891464DF5EACD
:10749300ED1DAE0470011C4E600FB1B170020566A4
:1074A30014F9120731F5E780E722789E7600087613
:1074B3000778A9E690878AF0C3742496FFE41896A8
:1074C300FED374079FEE6480F87480984007789E1B
:1074D300EEF608EFF6789EE6FE08E6FF78A8E6FCEF
:1074E30008E62422F974863CFA7B01788B7C8712A8
:1074F3004FDD7A87798A756A00756B087F017E0094
:10750300B126789EE6FE08E678A80826FFF618EE70
:1075130036FEF6C3EF9424EE648094804004E4F6D0
:1075230008F6228E658F668B678A68896943EB2824
:10753300E566640145657006B1A54002800CE56609
:1075430064024565700AB1A54006756A00756B084B
:10755300E478A0F608F6C378A1E6956BE56A648043
:10756300F5F018E6648095F0501CAB670569E56992
:10757300AA687002056814F9120731F5E60806E6F1
:107583001870010680D0E5EB648054804420FFE549
:1075930066640245657E0070027E40EF4E456BF5E2
:1075A300EB22D3E56B9408E56A6480948022AB6593
:1075B3000567E567AA6622908820E4F0A3F0A3F0AC
:1075C300908814F0A3F022908816E0FEB4210DA356
:1075D300E0B40908E490849DF07F0122EE64A17079
:1075E30023908817E0B4011C53EA7F7B017A8479E6
:1075F300DF7D087C0091799084DE7408F0FF1239F6
:107603009C7F01227F002275650175668875671668
:10761300E5ED540F6408600643EA407F0022E478F6
:107623009EF608F6B1B17002056614F9E5EF12078C
:1076330077789F06E618700106789FE66408184677
:1076430070E243ED807F01228B688A69896AE56C69
:10765300156CAC6B7002156B4C601D0FEFCCEECC50
:1076630070010E14F5828C83E0FDD17C70020569F4
:1076730014F9ED12077780D622AB68056AE56AAA8A
:10768300692290849CE06002E4F090841CE0600531
:10769300E4FF12399C2290883BE0FF20E70520E6B7
:1076A30002E1FD12377890883BE0FDC4540F9088C7
:1076B3003FF0ED30E71220E40720E5045430600882
:1076C30090883F7408F0C22090883BE0540F908864
:1076D3003DF0700204F07A2C7B6B752C03E4FD7F84
:1076E30002123354127810753219753382E4FB7D1C
:1076F30026123FB8127813753219753388E4FB7D6F
:10770300647F01124381300116752EFF752F1975A1
:10771300308B1257EEFD124F5E8E318F32800C7517
:107723002EFF752F197530921257DB7B027D1E7F5A
:107733000112438190883FE024FB7002E1C814608A
:1077430060146035146002E1F8127810753219750F
:107753003399127A12123FBA1278137532197533AC
:107763009F7B047D487F021243812020077F2212E2
:1077730079648073127913806E12781075321975DB
:1077830033A3127A12123FBA1278C57D6E7F0212AA
:1077930043812020077F21127964800312791380AB
:1077A300461278107532197533AF127A12123FBA36
:1077B3001278C5127B262020077F2012796480036C
:1077C30012791380221278107532197533B6127A32
:1077D30012123FBA1278C5127B262020077F1F1290
:1077E300796480031279131243167FC07EC67D2D00
:1077F3007C000250EF123778C220221208C7E4122D
:10780300038D7BDB7AF9791E783F020169752EFFC0
:10781300752F1975307F7531FF229087D5E0F532CA
:10782300A3E0F5339087BAE0FCA3E0FDA3E0FEA359
:10783300E02275321A75335C7B047D037F011243AA
:10784300817A2E7B68752C037D017F50123354C3DC
:107853007872E6946418E6940022E6FF7E00908432
:107863001FE02FF090841EE03EF0C3908421E09F40
:10787300FF908420E09EFEF0A3EFF04E22752EFFD2
:10788300752F137530897871E6F53108E6F5327B8B
:10789300032278711209A7EF2BFFEE3AFEED39FDB3
:1078A300EC38FC22EEFDE52C2DFDE433FC908768DB
:1078B300E07A002DFDEA3CFCD3ED947FEC648094E8
:1078C3008022752F197530AB90883DE0F5317B042C
:1078D30022E4FFFEFDFC78710209C42FF582E583E3
:1078E3003EF58322752EFF752F007530067531FF27
:1078F30075321A7533BDE4FB7D1E22A3E075F03C9F
:10790300A4FFEB2FFBEA35F0FAED39F9EC38F82256
:107913007F1B7EB0025631120074E4FBFA79707853
:10792300421202729087BA0209D090876CE08FF0FE
:10793300A4FF7875E6FC08E68C832FF58222F075A8
:10794300F080EDA42480F582E5F03480F583E582B0
:107953002F2275321B7533AF7B037D44E4FF024353
:10796300817EB0125631D22022E4FFFEFDFC9087C7
:107973003B0209D0F52E8E2D8D2C8C2B908803E0A5
:10798300F52F227D167F207E031236F078710209CF
:10799300C4E6FA08E6907FFE75F00A1209DCEA22D3
:1079A300E47871F608F608F608F69087E6E0227B9D
:1079B300017D0A7F02124381908400E0FD227878E2
:1079C300E62528FFE433FE08E6FD25292290875C9F
:1079D300E024FFF090875BE034FFF0221202721282
:1079E30003CB9087D5EEF0A3EF2212000EEF75F0D4
:1079F30006A4227531FF75321A7533B3E4FB7D1982
:107A030022788A1209C47C887D2FAF2BAE2A227B71
:107A130004E4FD7F022275F00AA485F031F53222D9
:107A230090880CE0FF7E007C007D0A227B1C7A3468
:107A330079CF78C10200781209A7D3020967EAFF58
:107A4300C3E52C9FFFE49400FE22F5831209B4746E
:107A5300F002031175321B7533AB7B03E4FF22087D
:107A6300E6FC08E6FDC39FEC9E2275F00AA478713C
:107A7300A6F008F622E47F107E0EFDFC90873722E5
:107A8300FED3EF947FEE64809480227531FF7532CC
:107A93001C75332B22E0FF7E00C37480948022FE8A
:107AA300A3E07873A60608F622752EFF752F1375CB
:107AB300303E22752EFF752F1375303422752EFF3D
:107AC300752F1275309B22E52B2408F582E4352AA5
:107AD30022E0FD5420FCED5480FA2275321A7533EE
:107AE300727B0322908839E0FEA3E0FF2275F00A3F
:107AF300ED1209DCEC2275F00AEB1209DCEA2290A4
:107B03008837E09087A4F0227871E6FE08E6FF4EFE
:107B1300229087F2E0908732F022908769F075F027
:107B230003A4227D647F020243817876E6FE08E6A1
:107B3300FF227873A60608A6072290880AE0FB7D39
:107B4300052290880CE0FB7D0622F9E43484FA7B5D
:107B530001227D32E4FF0243811234677B017D0100
:017B630022FF
:027FFE0014204D
:00000001FF
